:020000040800F2
:100000002A17002405030008A9020008A902000815
:10001000A9020008A9020008A9020008A902000814
:10002000A9020008A9020008A9020008A902000804
:10003000A9020008A9020008A9020008A9020008F4
:10004000A9020008A9020008A9020008A9020008E4
:10029000A9020008A90200080000000000000000F8
:1002A000FFECC2925D7D05C5EFF305801EF0040FE3
:1002B00002D0EFF309818D466A4602F16802EFF33E
:1002C00011831EF0100F0CBF2DED108A90B02DE998
:1002D000FC4F6946DFF828D000F044FAB0E8FC4F44
:1002E0001EF0100F0CBFB0EC108A40301EF0040F4F
:1002F0000CBF80F3088880F3098883F31188704766
:100300000003002408B5174A0021174B934221D35C
:10031000164B174A17498B421FD300F009F900F01A
:1003200039FA00F05BF9BFF34F8FBFF36F8F124ABA
:10033000136823F001031360536823F00103536033
:10034000BFF34F8FBFF36F8F00F068FC00F0F4F93C
:1003500000F076FC43F8041BD8E752F8040B43F88E
:10036000040BD8E73C140024000100240000002402
:1003700090A200080001002490EF00E0594B82B0E9
:100380001A6822F4802242F480321A60564A01929E
:10039000019A002A00F39F80019B002B40F3998073
:1003A000524A5349136823F4706323F00F0343F058
:1003B000080313600B6823F4E06343F040030B6011
:1003C0000B6823F4E06343F480630B60136823F04D
:1003D000700343F040031360936823F0700343F00D
:1003E00040039360434B444A283B9A62434A1A6352
:1003F000434A9A6302F500321A64424ADA621A6882
:1004000042F0A8521A601A689201FCD51A681001CD
:10041000FCD5344A13689900FCD53B4A136843F075
:1004200006031360394B1A6842F440421A601A6896
:100430009204FCD536490A689004FCD535490A680F
:1004400042F002020A6034490A6842F001020A607E
:100450001A689204FCD5314B22221A60304B1A687C
:1004600022F0070242F003021A601A6802F0380212
:10047000182AFAD12B482C4A036823F4405343F43A
:1004800000530360136823F4407343F40073136054
:10049000264B196821F4E04141F480511960196834
:1004A00021F4E02141F480311960116821F0E0412C
:1004B00041F080511160016821F4401141F40011B4
:1004C0000160116821F4403111601A6822F0405235
:1004D0001A6002B070471A6891033FF55DAF019A48
:1004E000013A54E70044025848BE2100184402581B
:1004F0001C440258284402581220200077020307A7
:100500002F0201018808BF000C4802581848025801
:1005100004480258F44402582C04005800200052A9
:100520001044025854440258584402585044025847
:1005300008B5204B012100201A6842F001021A6020
:100540001D4A11601D4A10601D4A19680A401D4964
:1005500042F010021A601C4A11601A6822F48022CC
:100560001A60186600F07AF8FFF708FF174A136858
:1005700043F0006343F001031360154B1A681A60DF
:1005800053F8082C43F8082C124A136843F08053A0
:1005900043F09F031360104B1A681A605A685A6040
:1005A0009A689A6053F8042C43F8042CDA68DA60ED
:1005B00008BD00BF00440258088100511044025891
:1005C00067EFFEEA0000FF012C440258D8440258AD
:1005D000DC440258E0440258E84402587047FFECFB
:1005E00030B4EFF3118400238022EFF3108372B64E
:1005F00082F3118883F31088BFF34F8F154B164A8F
:100600001B68118803F4807578B10131118012885C
:1006100075B1BAB10023BFF34F8FE4B284F31188F0
:10062000ABB1042030BC00F04AB849B10139EDE764
:10063000002AEFD043F48073064A13600123EAE7EF
:10064000002DE7D023F48073024A1360E2E730BC48
:10065000704700BF0048025800030024EFF31182E6
:1006600000238021EFF3108372B681F3118883F3A6
:10067000108806490B6823F480730B600021044B3B
:100680001980D3B283F31188FFF7AABF004802583C
:100690000003002430B5EFF3118400238025EFF32D
:1006A000108372B685F3118883F31088036823EAF8
:1006B0000101E3B20A43026083F3118830BD82B0C6
:1006C000002245F26161B0F57A7F0BD8002240F636
:1006D000A201642811D800220A2818D8002200BBE1
:1006E00002B070470192019B8B4202DDA0F57A7047
:1006F000E9E7019B01330193F5E70192019B8B42EE
:1007000001DD6438E5E7019B01330193F6E70192CF
:10071000019BDC2B01DD0A38DEE7019B01330193ED
:10072000F6E70192019B152B01DD0138D7E7019B0C
:1007300001330193F6E7FFECBFF34F8FBFF36F8FE9
:10074000064B00221A60064A136843F40033136014
:10075000BFF34F8FBFF36F8F704700BF50EF00E0C4
:1007600014ED00E037B50A4D0C462B680BB91C465A
:100770002960019000F0F3F82968019800F042FB2D
:1007800014B900232C682B60204603B030BD00BF95
:1007900004030024EFF3148343F0040383F3148869
:1007A000064A1368A2F5D67223F04043C2F8AC3172
:1007B000136843F470031360704700BF34EF00E028
:1007C0000F2810B531DDA0F110041F2C0ADC03F155
:1007D000604303F561430B60012303FA04F41460E2
:1007E00000201CE03F2C08D81C4C30381C440C6006
:1007F000012303FA00F01060F2E75F2C04D8184CD4
:1008000050381C440C60F3E77F2C04D8154C70382A
:100810001C440C60ECE7952C02D94FF0FF3010BD62
:10082000114C90381C440C60E2E7104B04280B601C
:1008300003D14FF480331360D2E7052802D14FF47F
:100840000033F8E7062802D14FF48023F3E70F289E
:10085000E3D1074B0B600123EDE700BF04E100E0AB
:1008600008E100E00CE100E010E100E024ED00E030
:1008700010E000E01D4B4FF0FF301D4910B51B6824
:1008800003F00F035A1C03F1382361339B0041F836
:10089000040B8B42FBD1174B1749184C19604FF0D2
:1008A00080311961216099615301154A03F1604358
:1008B00003F5644342F8041B9342FBD1114B002221
:1008C00011490B201A6000F075FA00220F4903202D
:1008D00000F070FA236823F07F4343F0E043236085
:1008E000F02383F3118862B610BD00BF04E000E07E
:1008F00080E100E008ED00E0000000081CED00E0F1
:1009000000E400E0040300249509000861090008E0
:1009100013B5802301AA69460446FFF751FF20B9A9
:100920000F2CDDE9003102DD196002B010BD1A683C
:1009300022EA01021A60F8E713B5002301AA69460A
:100940000446FFF73DFF20B90F2CDDE9003102DD41
:10095000196002B010BD1A680A431A60F9E77047BF
:1009600008B5094B1B68094B1B68EFF31183002383
:100970008022EFF3108372B682F3118883F310881C
:10098000AD21034800F03CF92CED00E028ED00E03B
:10099000909C0008CA6E012A08B508D0022A0AD025
:1009A0001AB9D422086F00F023F8002008BD0A6F9E
:1009B000034B1A60F9E70A6F11604A6FF8E700BF4E
:1009C00004030024FFECC2925D7D05C5FFECC292DA
:1009D00018DF88DFCD06CD767CD30CD3D982D9122F
:1009E0002C00050A0F14191E232800BFAFF3008046
:1009F00000B501B400F004F801BC00BDAFF3008005
:100A000000B5042A60DB00F0030E61F3830E7A4B1D
:100A1000D3E80EF0AFF30080AFF30080AFF30080B7
:100A200011F8013B00F8013BA2F1010211F8013B72
:100A300000F8013BA2F1010211F8013B00F8013B73
:100A4000A2F101022DE9F01F282A07DBB1E8F81F07
:100A5000A0E8F81FA2F12802282AF7DADFF89CE1C3
:100A60004FEA920BDEE80BF051F8043B40F8043BF0
:100A700026E0B1E81800A0E8180021E0B1E838004D
:100A8000A0E838001CE0B1E87800A0E8780017E0A2
:100A9000B1E8F800A0E8F80012E0B1E8F801A0E839
:100AA000F8010DE0B1E8F803A0E8F80308E0B1E8C8
:100AB000F807A0E8F80703E0B1E8F80FA0E8F80F9E
:100AC000BDE8F01F02F00302002A08BF00BD11F8C4
:100AD000013B00F8013B013A08BF00BD11F8013BA2
:100AE00000F8013B013A08BF00BD11F8013B00F8D6
:100AF000013B00BDAFF30080AFF30080AFF3008097
:100B000011F8013B00F8013BA2F1010211F8013B91
:100B100000F8013BA2F1010211F8013B00F8013B92
:100B2000A2F10102282A35DB2DE9F01FB1E8F81FF8
:100B300020F8023B4FEA134364F31F434FEA144487
:100B400065F31F444FEA154566F31F454FEA164605
:100B500067F31F464FEA174768F31F474FEA1848E5
:100B600069F31F484FEA19496AF31F494FEA1A4AC5
:100B70006BF31F4A4FEA1B4B6CF31F4BA0E8F80FB7
:100B80004FEA1C4C20F802CBA2F12802282ACDDA29
:100B9000BDE8F01F042A97DB51F8043B20F8023B24
:100BA0004FEA134320F8023BA2F10402BAE711F81E
:100BB000013B00F8013BA2F1010211F8013B00F8F2
:100BC000013BA2F1010211F8013B00F8013BA2F147
:100BD0000102042AFFF678AF51F8043B00F8013B0C
:100BE0004FEA132320F8023B4FEA134300F8013B7E
:100BF000A2F10402EDE70000D0090008E0090008B6
:100C000008B501F07DFB012000F004F8012008B5D3
:100C100000F000F808B500F03DFB704700F008B8A0
:100C2000002070470021084601F018BA04F07ABD90
:100C3000014801F065BA00BF080C02007047FFECE4
:100C40003C4C01233C4D8C2204F170062B7083B583
:100C50000021204603F0FEFD0323182237492377A5
:100C60003046374B374FC4E905330623E38303F09F
:100C700040FE354920463E6003F0F9FB334B01A9A5
:100C80006846334E1C6002232B7001F017FADDE931
:100C9000000103F0FBF9042333603368012B45DDC9
:100CA0003068800003F010FA2A4B18603368046043
:100CB0002048A17F00F00AFBA3681E48DB685F6044
:100CC00001F072FC1B4800F0F3FA1A4800F01CFB1C
:100CD000A36805221A7200221F4B1A6003232B708F
:100CE00000F0C0F806F074FD1C4B0BB100F034FBB3
:100CF0001B4B0BB107F08DFB1A4B0BB100F082FFC1
:100D000001F0AAF901F090FB05F043F8042309482B
:100D10002B7000F01CFB05232B7000F039F8062324
:100D20002B7000F0AFF801F03DFCFCE733685B008E
:100D3000B2E700BF10030024AC030024A89C000805
:100D4000410C000808030024BC030024C403002451
:100D5000A8030024B8030024A403002459130008A6
:100D600013840008051C000813B50024FFF75AFF80
:100D7000054B4FF4386264210094044800F0D9F820
:100D8000204602B010BD00BFE1950008F49C0008A9
:100D900013B50024054B4FF40062FE210094044873
:100DA00000F0E0F8204602B010BD00BF690D000859
:100DB000049D0008A52870B505460C461AD8EFF327
:100DC000118600238021EFF3108372B681F311881E
:100DD00083F310881CB9FFF79BFD2246074C084897
:100DE000F6B240F8354000EBC500426086F311884A
:100DF000002070BD6FF01500FBE700BF410E00083A
:100E0000E0030024A52808B50CD8094A52F8303070
:100E10005BB102EBC00252689847064B1A68064B5A
:100E20001A6008BD0022054BF6E71A46FBE700BF33
:100E3000E0030024BC030024C4030024410E000886
:100E400008B5EFF3118300238022EFF3108372B60D
:100E500082F3118883F3108836210148FFF7D0FE12
:100E60000F9D0008054B1B682BB1054A126812B98B
:100E70001A8C01321A840020704700BFBC03002482
:100E800004030024134B10B51A68C2B1124B1B683F
:100E9000ABB9EFF311848021EFF3108372B681F3C5
:100EA000118883F31088B2F92030002B09DC00236D
:100EB00013840A4B1B6853B9E4B284F311880020F1
:100EC00010BD013B9BB21384002BF5D1EFE701F07D
:100ED000C3FAF1E7BC03002404030024B003002498
:100EE00070B586B005468C200E46CDE9043203F07D
:100EF000EBF80446D0B10021C68303910C9902910E
:100F00000B9901910A99DDE904320091294600F01C
:100F100033F8051E05DA204603F0C6F8284606B069
:100F200070BD2046E56800F079F9F7E76FF00B0532
:100F3000F4E71FB5069C00920A46CDE90134002370
:100F40001946FFF7CDFF04B010BD1FB5079C0294F2
:100F5000069CCDE9003413460A460221FFF7C0FF84
:100F600004B010BD13B5049CCDE900341346002233
:100F7000FFF7EBFF02B010BD2DE9F347867F8846EF
:100F80000546914631461F46DDF828A000F09EF93F
:100F9000041E3ADB284606F0030600F0DAF9041EC8
:100FA0000CDB87B152463946284601F0C3FA041ECD
:100FB00005DB284600F07CF9041E13DA57B12846F9
:100FC00000F0A8F921E032465146284601F0EAF93E
:100FD000041EEEDAAB6B002BF1D03146284601F04F
:100FE00055FAECE70B9B49460A4A2846009600F062
:100FF00013F8041EE2DB0C9A4146284600F0A2F8E2
:10100000041EDBDB284600F07FF9204602B0BDE875
:10101000F08700BF411200082DE9F74F04460E4645
:10102000CDE90023EFF3118700238022EFF3108333
:1010300072B682F3118883F31088DFF800A1DFF81D
:101040000081D346DAF800500020D8F800100135AE
:10105000384A136898420DDB1068C00003F034F87A
:10106000344A0546002846D1FFB287F311886FF055
:101070000B003AE0012D1368B8BF0125013B2B405E
:1010800051F8239001EB830EB9F1000F30D1CEF867
:101090000040FFB2E560CBF8005087F31188E28B87
:1010A000F6B29DF830100320009B22F0630201F09D
:1010B0000301267463610A43019B49466674A36178
:1010C000E28304F1440200F083F9204684F81C9086
:1010D00001F06AFAFFF7C6FE1749204603F0C7F988
:1010E00004222277FFF7CEFE484603B0BDE8F08F1A
:1010F00001350130ADE713680E495B001360002233
:101100000B68D8F8000003EBD373B2EB630F04DB7A
:1011100002F0CAFFC8F8005094E750F822000132EC
:101120000B6803F1FF3EC3680EEA030345F8230092
:10113000E6E700BFA80300249C030024A4030024C6
:10114000B8030024344B2DE9F74F002914BF88461B
:10115000984607460024154641461822703003F091
:10116000ECFB404687F8884003F0DFFB461C4DBB94
:101170002C460234384606EB840101F099F9064604
:101180004FEA8409002844D000EB090AA9F10809B4
:10119000B346043DC0F800A0404603F0C6FB044639
:1011A000B14441460134504603F09BFB5444D945B9
:1011B0001BD100204AF8040CBA68D268566003B00C
:1011C000BDE8F08F40F2011955F824000028D0D076
:1011D00003F0ABFB01307B6B06449E4216D2013418
:1011E0004C45F1D16FF00600E9E74BF8044F55F894
:1011F000041F0846019103F098FB804601992046A0
:1012000008F1010803F06DFB4444D0E76FF05A0089
:10121000D5E76FF00B00D2E7279D000810B5EFF37C
:10122000118400238022EFF3108372B682F31188B9
:1012300083F3108801F060F9E4B284F3118810BDE3
:1012400038B5134B1C68E38B03F00303022B02D069
:10125000204600F0ABFBA368012040F20111DB68DF
:101260005A6852F820304BB9E38BA56903F00303A9
:10127000022B08D11146A847FFF7CCFC0130884269
:10128000EFD10120F8E70146284603F009F9F8E715
:10129000BC0300240446002208B5E4B2034B2146F7
:1012A000186800F0ABFB204601F0A2F8BC03002454
:1012B00010B51821044601F0FBF820B1A368DB68E3
:1012C0000360002010BD6FF00B00FBE770B5064611
:1012D0004FF48E7002F0F8FE044690B100F0B3FBBC
:1012E000051E04DA204602F0DFFE284670BD04F138
:1012F0002400B46006F09DFA2046002503F0DEF9D4
:10130000F3E76FF00B05F0E7D0E902321A60012233
:101310005A72704738B58468054634B1637A012B38
:1013200004D9013B63720023AB6038BD204600F056
:101330009BFB204600F032F904F1240006F07DFA10
:10134000204603F0DAF9204602F0AEFEEBE700F0AB
:1013500098BB00F096BBFFEC0023044A044942F816
:1013600033100133A62BFAD1FFF784BAE00300242F
:10137000410E000838B5044618B3C068B0B1EFF3A9
:10138000118200238025EFF3108372B685F3118854
:1013900083F310880C4B00251B68013B03400B486E
:1013A000006840F82350D3B283F31188A36B13B1C4
:1013B000204601F06BF82046FFF7ACFF204602F014
:1013C00073FE002038BD00BFA8030024B80300242A
:1013D000F8B51746194B06460C461D68FFF742FD47
:1013E0000FB16B6C3B60D4B1EFF31183002280210D
:1013F000EFF3108272B681F3118882F31088022E07
:1014000011D0032E14D0012E14D16A6C21680A4326
:1014100000246A64DBB283F3118800F011F8FFF74F
:1014200031FD2046F8BD21686A6C22EA0102EFE72F
:101430002268EDE76FF01504ECE700BFBC03002461
:10144000184B30B51D6885B0FFF70CFD6C6C284655
:1014500000F000FDE4430440039424B9FFF712FDBB
:10146000204605B030BD03A800F070F8431C0146CB
:1014700010D0019003A803F05DF80199284600F010
:1014800013F8044630B1011D284600F09BF82046B1
:1014900000F02EF8039B002BE5D1FFF7F3FC0120B1
:1014A000DFE700BFBC03002438B58368EFF3118584
:1014B00000228020EFF3108272B680F3118882F34D
:1014C000108800209C6974B122798A4206D103F108
:1014D000180130B9084602F0A5FF04E02046246850
:1014E000F1E702F0A9FFEDB285F31188204638BD7F
:1014F00010B5037B83B9EFF311848022EFF31083DF
:1015000072B682F3118883F310880E4902F06AFFE5
:10151000E4B284F3118810BD022B0CD1EFF31184D7
:1015200000238022EFF3108372B682F3118883F3D5
:1015300010880549EAE7012BEDD1BDE8104002F023
:10154000B3BD00BF300900242809002438B5054682
:1015500001242146284602F0FEFF20B90134202C48
:10156000F7D14FF0FF34204638BD38B5044600F1BE
:101570004C05284602F056FF50B904F154052846A0
:1015800002F050FF38B94FF0FF32C4E9112038BDE6
:1015900000F0BAFCEDE700F0B7FCF0E738B5044620
:1015A00000F11005284602F03DFF28B91834204606
:1015B00002F038FF18B938BD00F082FBF2E7FFF700
:1015C00097FFF4E72DE9F0410D460978044629B369
:1015D000443002F0C0FF012807467ED1EFF31186A8
:1015E00000238022EFF3108372B682F3118883F315
:1015F0001088237FF6B2062B12D1297804F1480017
:1016000002F0A9FF60B12B682046E3656B68236692
:101610000023A36400F070FF86F311880026B4E075
:1016200086F31188A4682978EFF3118200238020C3
:10163000EFF3108372B680F3118883F31088A369E7
:1016400013B11879884208D1D2B282F3118833B12C
:101650002A685A606A689A60E0E71B68F0E7564BB0
:101660001B68FBB1554802F0DDFE20B9544802F07A
:10167000D9FE0028D2D02B6843606B688360EFF3FB
:10168000118500238022EFF3108372B682F3118854
:1016900083F3108804F11801EDB202F0A3FE85F384
:1016A0001188BBE7EFF3118600238022EFF310834C
:1016B00072B682F3118883F310884048F6B202F0C4
:1016C000B1FE86F311880028D5D1102002F0F4FC79
:1016D0000028A3D001230373CDE7FFF7C3FB2978CC
:1016E000A06800F0D3FB064600282CD0406848B321
:1016F00000F0DEFB00284BD073684360B268826064
:10170000F3689B0604D4297801238B40134383603C
:101710002B68C3606B680361EFF31186002380229E
:10172000EFF3108372B682F3118883F3108804F10B
:101730004C01F6B202F056FE2249204600F070FF3E
:1017400086F311880026FFF79DFBEFF31188002335
:101750008022EFF3108372B682F3118883F310882E
:10176000237F062B08D12B682046E3656B68236630
:101770000023A36400F0C0FE5FFA88F888F31188A4
:10178000002F08D001DA6FF015063046BDE8F08171
:101790006FF00B06D7E7237F052B03D104212046EA
:1017A00000F012FA237F072BEFD12B78082BECD116
:1017B000204600F0C6F9E8E70403002430090024BD
:1017C00028090024E917000807B5019100F072F913
:1017D00028B1019903B05DF804EBFFF7F3BE6FF099
:1017E000020003B05DF804FB2DE9F04F87B004461A
:1017F00002F0EEFD03684FF0800904F14C0A0193FA
:1018000004F15408B4F922300293EFF31183039FDB
:10181000EFF3108772B689F3118887F31088E28B93
:101820000397DFB212F400720AD087F3118802F036
:10183000CFFD019B0360029B638407B0BDE8F08F7E
:101840005046059202F0EEFD059A06460028ECD0BF
:10185000E18B059241F40071E183414602F0C2FD43
:10186000D4F844B0B5684BEA0505656487F3118880
:10187000736806F10C01059A307B9847EFF31183EA
:10188000049A0593EFF3108272B689F3118882F3FC
:10189000108804924146E28B304622F40072E283C3
:1018A000626C554082EA0B02154085EA0B056564BF
:1018B00002F0A2FD059BDBB283F31188FFF7C0FDA8
:1018C000304600F021FBA0E77047FFEC054B10B558
:1018D0001C68FFF7C7FA204600F012F9BDE8104077
:1018E000FFF7D0BABC03002408B5024B01201B68E7
:1018F000FFF790F9BC03002408B58068203002F09F
:101900002AFE0028D4BF0020012008BD0023084A79
:1019100012F83310814206D102EBC3035878C0435A
:1019200000F00100704701330B2BF1D1012070470B
:10193000309D000838B585685AB100231A4A12F85C
:101940003300814219D102EBC30305F120005C682A
:10195000BCB9EFF3118400238022EFF3108372B639
:1019600082F3118883F3108805F12000E4B202F0BD
:10197000E1FD84F31188002413E001330B2BDED149
:10198000E7E7EFF3118500238022EFF3108372B6AF
:1019900082F3118883F3108802F0BFFDEDB285F366
:1019A0001188204638BD00BF309D00082DE9F04366
:1019B00086680024104D4FF002092036A04685B0FD
:1019C000304602F0C4FD6B6873B12F7801A9002284
:1019D000CDF80C903846CDE90138012300F086F9A6
:1019E0003946304602F099FD013408350B2CEAD116
:1019F000002005B0BDE8F083309D000810B5C38B12
:101A000004461B0515D43AB9806828B1437A012BE6
:101A100002D12C3002F0BCFD204600F00BF820462D
:101A2000FFF778FC2046FFF7A0FDE38B43F400634B
:101A3000E38310BD10B5044600F020F82046BDE851
:101A4000104000F0A8B838B50546382002F03CFB3D
:101A5000044630B10122002102F02DFD0020EC608F
:101A600038BD6FF00B00FBE710B5C468204600F0EE
:101A70007AF82046BDE8104002F016BB243000F092
:101A800071BA002307B5024601900121184606F0FD
:101A90009FFB019A00230621012006F099FB0023F9
:101AA000019A0621022006F093FB002003B05DF8A6
:101AB00004FBFFEC0346EFF3118100228020EFF3DB
:101AC000108272B680F3118882F310880A4A106877
:101AD00060B1002B0EDB094A1268013A1A4050F837
:101AE000220018B1C2689A4218BF0020CBB283F31B
:101AF000118870470020F9E7B8030024A8030024E8
:101B000038B50446EFF3118500238022EFF31083EC
:101B100072B682F3118883F31088037F043B032B92
:101B20000BD800F067FA042307212046638400F0F5
:101B30004DFAEDB285F3118838BD072100F006FC9F
:101B4000F7E710B5EFF3118400238022EFF3108341
:101B500072B682F3118883F3108800F0CDFCE4B2F2
:101B600084F3118810BD30B103881B0401D4012314
:101B70000380002070476FF01500704710B5FFF725
:101B8000F2FF041E05DA644202F022FC04604FF00A
:101B9000FF34204610BDEFF3118200238021EFF3C4
:101BA000108372B681F3118883F31088037F052BAD
:101BB00006D1016C0B8801331BB20B800023036438
:101BC000D3B283F31188704738B5EFF31184002244
:101BD0008025EFF3108272B685F3118882F31088A6
:101BE000027F052A09D1056C2A88013212B22A80A7
:101BF00000224184026400F07FFCE4B284F3118887
:101C000038BDFFECF8B50024284B294E6020C3E90D
:101C10000044284BC3E90044274BC3E90044274B49
:101C2000C6E90044C3E9004402F046FA054648B15B
:101C300000F160072C7528461835314602F0D2FBBA
:101C4000AF42F7D1602002F037FA044658B100F1F4
:101C500060050227174E277520461834314602F0DA
:101C6000C1FBA542F7D1402002F026FA044658B144
:101C700000F140050027104E2773204610343146EE
:101C800002F0B0FBA542F7D1402002F015FA04465D
:101C900058B100F140050227084E27732046103442
:101CA000314602F09FFBA542F7D1F8BD1009002490
:101CB00018090024200900243009002428090024E0
:101CC00010B5EFF3118400238022EFF3108372B676
:101CD00082F3118883F310880349E4B202F082FB97
:101CE00084F3118810BD00BF100900242DE9F04FC6
:101CF0001546564A1F2885B0D2F800B007460E4652
:101D0000DBF808A004D96FF0150005B0BDE8F08F2E
:101D100041B93946504600F0B9F8044665B916BBDA
:101D20000020F2E7002BF4D10B68012BF1D0FFF774
:101D3000EDFD0028EDD1E6E739465846FFF7DCFD1A
:101D400030B100230122C5E900230223AB60E6E79E
:101D50002CB163682B60A3686B60E368F6E7C5E9A4
:101D60000044AC60DBE73568012D11D12A463946C5
:101D70005846FFF7DFFD054685B9002CD0D0204638
:101D80000AF1100102F038FB2046FFF799FFC7E780
:101D9000002239465846FFF7CDFDEDE7ECB9EFF3E9
:101DA000118B80220023EFF3108372B682F3118827
:101DB00083F31088264802F035FB04465FFA8BF364
:101DC00083F311888022DFF888B001925CB10AF1B8
:101DD00010012046277402F005FB65607368A3605C
:101DE000B368E3609CE7502002F066F90446C8B18E
:101DF000EFF31183019AEFF3108972B682F3118821
:101E000089F3108800F15002204659461434CDE978
:101E1000022302F0E7FA029A039B9442F4D1DBB268
:101E200083F31188EFF311830293019BEFF3108882
:101E300072B683F3118888F31088584602F0F2FADC
:101E4000029B0446DBB283F31188BFE7BC03002486
:101E500010090024002337B582680193EFF3118540
:101E60008021EFF3108372B681F3118883F3108819
:101E700094692CB9EDB285F31188019803B030BD97
:101E8000217901A802F049FB2468F2E738B50D4634
:101E9000044640B1FEF7E6FF246914B1237CAB424F
:101EA00003D1FEF7EFFF204638BD2468F5E7FFECCD
:101EB000124B10B51B6843B1114802F0B3FAE0B9F8
:101EC0001048BDE8104002F0ADBAEFF311840023D2
:101ED0008022EFF3108372B682F3118883F31088A7
:101EE0000748E4B202F09EFA84F3118828B918205A
:101EF00002F0E2F808B10123037510BD04030024C9
:101F0000180900242009002410B5037D83B9EFF3DC
:101F100011848022EFF3108372B682F3118883F369
:101F200010880E4902F05EFAE4B284F3118810BD05
:101F3000022B0CD1EFF3118400238022EFF31083E6
:101F400072B682F3118883F310880549EAE7012B02
:101F5000EDD1BDE8104002F0A7B800BF1809002479
:101F60002009002438B50446EFF3118500238022B0
:101F7000EFF3108372B682F3118883F31088F0B107
:101F80004368E3B1104B00201B68DBB1A3420FD1C3
:101F900023681BB19A68A1680A449A6058B10A493B
:101FA00002F04AFA00206060EDB285F3118838BD76
:101FB00018461B68E9E7044802F034FAF2E76FF0CC
:101FC0001500F1E71B68FFDE3809002438B50C4620
:101FD000074B054653F8311003EBC4031B79DB07AD
:101FE00003D500F015F82C7738BD02F035FAFAE782
:101FF000B49C0008054B027F10B553F8321004461C
:1020000002F040FA0023237710BD00BFB49C000803
:1020100010B50B68027CB3B11C7C944206D25A689E
:1020200062B9C0E900325860086013E01B68F2E74B
:10203000C0E900321060486000200CE0C0E90032C6
:1020400010605860F8E74A68002AF1D1C0E900330F
:10205000C1E90000012010BD7047FFEC37B5124DFB
:102060002C682CB1114802F080FA012003B030BD79
:102070000F4802F07AFA40F2011369464FF60C70ED
:10208000ADF800308DF80240019503F049FE011EC5
:1020900004DA4942074802F068FAE6E7064802F027
:1020A00064FA2046E2E700BF40090024889D00084A
:1020B000AB9D0008D69D0008159E0008044B1B68C8
:1020C0000360C3F1105303F500230B60704700BF9A
:1020D0008C9C000802064FEA10130CD403F00F0387
:1020E000064A52F8232032B100F00F00012319B143
:1020F00003FA00F0906170471030F9E7509E000835
:102100002DE9F04705090446C0F3031715F008054B
:1021100040F0D3806A4B53F82760002E00F0CD804A
:1021200000F4402300F00F08B3F5002F00F0B28058
:10213000B3F5402F00F0B080B3F5802F40F0AE80B3
:10214000C0F30021FFF7C6FF0121EFF31182002346
:102150008020EFF3108372B680F3118883F3108828
:10216000022940F09D8014F4704FC4F3033017D05F
:1021700023074FF00F094BBFA8F1080343464FF068
:10218000240C4FF0200C9B005CF806E009FA03F9E0
:1021900000FA03F32EEA090E43EA0E034CF8063068
:1021A0004FEA48090323D6F800E0032903FA09F3AC
:1021B0002EEA030E6FEA030C01FA09F343EA0E0359
:1021C00033606FD004F44033B3F5803F6CD0B3F587
:1021D000003F0CBF02230023D6F80CE003FA09F3FA
:1021E0000CEA0E0E43EA0E03F36080B923074FF0AA
:1021F0000F0A4BBFA8F108034346242020209B0070
:1022000050F806E00AFA03F32EEA0303835101F1C2
:10221000FF3EBEF1010F0DD804F44065B5F5006F27
:1022200044D0B5F5406F43D0A5F5806ADAF10005DA
:1022300045EB0A05B36805FA09F50120BEF1010F67
:102240000CEA030C00FA08F045EA0C05B560736867
:1022500030D8A5052ED503430129736014D0E305BA
:1022600012D504F00C044FEA88030F2004F1B044A7
:1022700003F00C03D4F80814984007FA03F321EA9A
:1022800000010B43C4F80834D2B282F31188002055
:10229000BDE8F087022158E7032156E7294654E7B5
:1022A00000207DE7002397E7012395E70225C1E79A
:1022B0000325BFE723EA0003CEE76FF01500E7E749
:1022C000509E0008C0B2FFF71BBFFFEC02064FEAAA
:1022D000101310D403F00F03084A52F8233053B1FF
:1022E0001A6900F00F00012303FA00F0104214BF36
:1022F0001846002070470020704700BF509E00081D
:1023000008B504F0BDFA04F0BBFA04F0B9FA0D4BBD
:10231000186818B90C4B1B681B6873B9002007F0CC
:1023200035FAEFF3118300238022EFF3108372B6A6
:1023300082F3118883F31088FEE7BDE8084007F0B8
:1023400025BA00BF04030024BC030024F7B50646E9
:10235000114D01912F6806F093F80199044630461B
:10236000FFF734FE0D4B1B681BB106F09DF82043B0
:10237000C4B234B10A4B1A682AB1FA662A68D26E1E
:102380001A6003B0F0BD2B6807F16C00D96E03B082
:10239000BDE8F04000F0A7B8BC030024B00300245F
:1023A0000403002438B5836B0C46054611469BB9DF
:1023B000204601F081FEA863A86BB0B10119E86363
:1023C00021F00701091A696300F0CCF8EB8B0020BB
:1023D00043F48053EB8338BD436BA342ECD000F051
:1023E00055F8AB6B002BE7D1E2E74FF0FF30F2E797
:1023F000094C08B52368EFF3118300238022EFF323
:10240000108372B682F3118883F3108806F0A4F962
:102410002368D86E00F002F8BC03002401460120B6
:1024200000B500DF5DF804FB08B5084A80230849C1
:10243000013B42F8041BFBD1064B0BB1AFF300800C
:1024400000F078FBBDE8084001F0B0BC00010024BA
:10245000EFBEADDE0000000038B50A4C256806F07E
:1024600023F830B1084B1A6822B1EA662268D26EAE
:102470001A6038BD236805F16C00D96EBDE838409C
:1024800000F031B8BC0300240403002410B5044656
:10249000806B20B1E38BDB0401D501F005FEE38BFB
:1024A00023F48053E3830023C4E90E33636310BD38
:1024B00038B50731836B044621F007057BB1436BC8
:1024C000AB420ED9C36B2A460021184602F0C2F96E
:1024D000E26B03462A44E263626B521B6263184656
:1024E00038BD0023FBE703460A460220194600B523
:1024F00000DF5DF804FBFFEC70B505460B4C266869
:10250000FFF778FD284605F097FF30B1084B1A68B1
:1025100022B1F2662268D26E1A6070BD236806F19D
:102520006C00D96EBDE87040FFF7DDBFBC0300242E
:102530000403002470B5836B06460D46144623B190
:10254000817F01F00301FFF7A1FF2C44284624F00E
:102550000704611BC6E90E55716300F003F8002003
:1025600070BDFFEC90B5C41D83B024F0070400AF2C
:10257000224679B9391DB94228BF394621F00703EF
:10258000191A074B21F0030121448A4204D10C3768
:10259000BD4690BD0144F1E742F8043BF5E700BFBA
:1025A000EFBEADDE7047FFEC38B50025C1680446CC
:1025B00045668566C56661B9184B186840F2EE231A
:1025C000A0F2EE206363C4E90E00BDE83840FFF7D7
:1025D000C9BF406BD4222946A0F1D403E06B184454
:1025E000E06602F037F9E36B616BE26E0B44136057
:1025F0006369E26E23F00103C2F884304FF0807209
:10260000E36EC3F888206FF01602E36E9A62F02240
:10261000E36EC3F8CC50E36E5A6038BD8C9C000862
:1026200010B5436E044603BB1B4B1A6882421DD192
:102630001A4C236813B9BDE810400847A3F1D40031
:10264000C2E91913D42219462060FEF7D1F9236894
:1026500003F1D4021A60124A2368C3F8842080224E
:102660005A604FF08072C3F8882010BD4166D422B2
:10267000C16E8166A1F1D400E066FEF7B9F9E36EA0
:1026800003F1D4021A60064AE36EC3F88420802264
:10269000E36E5A60E36EE4E7BC0300240403002405
:1026A000A526000838B50D4B1C68F023A56E83F3F2
:1026B000118862B6636E20469847EFF311830023BA
:1026C0008022EFF3108372B682F3118883F31088AF
:1026D000002328466366FFF7A1FE00BFBC03002469
:1026E00010B5846E01F4D873A0F8501001F0010108
:1026F000226822F4D87213432360826E936823F019
:1027000001031943916010BD10B5EFF3118400234C
:102710008022EFF3108372B682F3118883F310885E
:10272000FFF7DEFFE4B284F3118810BDF0B5C36B90
:10273000EFF3118400228021EFF3108272B681F34F
:10274000118882F31088996E0A6822F0010002F065
:1027500001050860DE6D5F6E710801EB4701B1FB9A
:10276000F6F164293AD9013122F40040490820F0F9
:1027700001009A6E10609A6ED16093F85610234A49
:10278000012902EA000233D142F4C06293F85700F3
:10279000092802D0082830D179B342F48052996ECA
:1027A0000A60986E93F85860416821F440510EB168
:1027B00041F400514160986E93F85960816821F4AA
:1027C00040711EB15E6F0EB141F4807181602A4389
:1027D0009B6EE4B21A6084F31188F0BDC1F342022B
:1027E00021F00F0140F400400904090C1143C0E737
:1027F000022908BF42F48062C8E7B3F85610B1F569
:10280000E06F08BF42F08052C9E700BFFEE9FFEF6A
:10281000C36B9A6E506AB3F8522040EA0242C0B2CB
:102820000A600022A3F85220704710B5C06BEFF386
:10283000118400238022EFF3108372B682F3118893
:1028400083F31088B0F8503039B143F02001E4B27E
:10285000FFF75AFF84F3118810BD23F4907121F023
:102860000101F4E7C36B9B6ED869C0F34010704759
:10287000C36B9B6E9962704710B5C06BEFF3118408
:1028800000238022EFF3108372B682F3118883F362
:102890001088B0F8503041B143EA020189B2E4B285
:1028A000FFF732FF84F3118810BD23F08001090483
:1028B000090CF4E7C36B9B6ED869C0F3C010704776
:1028C00038B583685D6940F201139942EC6B05D01D
:1028D000B1F5817F29D06FF0180038BD002A4CD0A7
:1028E00094F85630FBB1012B4FF480710CBF4FF4BC
:1028F000007300230B4394F858101046002914BFAE
:10290000402100210B4394F85910002914BF4FF0C7
:10291000004100210B4343F030039360E16D02F06E
:102920001FF80020D9E71946E4E732B3936803F0B3
:102930003001302921D1002B01DA616FE9B113F4A4
:10294000807117D013F4007F14BF0123022384F891
:10295000563093681046C3F3801384F85830936858
:10296000DB0F84F8593002F01BF8E0652846FFF7CA
:10297000DDFED6E784F85610EBE76FF01500ACE704
:1029800010B5C46B94F86000FDF7C2FF002294F804
:1029900060001146BDE81040FEF70CBA38B5C56BB3
:1029A00006492A4695F86000FEF704FA044618B96D
:1029B00095F86000FDF7C0FF204638BDE12900080A
:1029C00010B5C36B144693F859302BB1836B9B69D8
:1029D00022B1002198472346184610BD0121F9E78E
:1029E00010B51446926ED3699BB29806A4F8523083
:1029F00013D5B4F8501089060FD5204603F0ECFE2D
:102A0000B4F852301A0606D5B4F850301B0602D579
:102A1000204603F0ABFE002010BD13F00E0FEFD0E8
:102A20000E231362ECE7FFEC38B5C46B00210546BA
:102A3000A36E1960C36B9A6E1E4B9A4204D14FF479
:102A400080221D48FDF726FEE06EFFF759FB206F40
:102A5000FFF756FB606F08B1FFF752FBA26E94F8C8
:102A60005810536823F47D5309B143F40053536065
:102A70002846A26E114B11680B401360A26E94F8A9
:102A80005510936823F4E06323F0010343EA4163A4
:102A90009360FFF74BFEA26E0020136843F00053D3
:102AA00043F00D0313600123A4F8500084F8543060
:102AB00038BD00BF00480040E844025803BEFF3361
:102AC000F8B50026C46B054684F85460EFF311870F
:102AD00080223346EFF3108372B682F3118883F3BA
:102AE000108831462046FFF7FBFDFFB287F31188BF
:102AF000EB6B9A6E0D4B9A4205D132464FF4802112
:102B00000B48FDF7C7FDA26E136823F00D03136099
:102B1000E06EFFF7D7FB206FFFF7D4FB606F18B1B3
:102B2000BDE8F840FFF7CEBBF8BD00BF004800404D
:102B3000E84402587FB50B49684601F0D2FE0023F5
:102B4000094D1C4655F8041B39B15E1C30336846EC
:102B50008DF8093003F020FC33460134082CF1D104
:102B600004B070BD709E00087C9E0008704738B5A8
:102B70000A460169044629B14B69036103B94361FF
:102B800000234B61637E207EC3F3C00520B9E0685B
:102B9000007C60F3C3036376CB6820464A81984784
:102BA000637E65F3C303637638BD37B50446C068FA
:102BB0000A4680B10368B4F85E10009121469D6812
:102BC00004F11D03A847002803DA237C43F0010326
:102BD000237403B030BD6FF00400F6E7F0B5047E57
:102BE00034B313466401144FE5592E0415D4AE03D3
:102BF000124E48BF45F080652E40334343EA81437F
:102C000001F04F0143F0805343F40043E351437E0E
:102C1000C28023F04F0319434176037E0020084908
:102C200003F1100201230C68934023430B60F0BDB5
:102C300021462346D6E700BF000B084000F8F3FF0B
:102C40001C080840E0B590F818C0134E4FEA4C1726
:102C5000BD592B0417D4AB03104B48BF45F080651A
:102C60002B40134343EA814301F04F0143EA8C5365
:102C700043F0805343F40043BB51437EC28023F0B2
:102C80004F0319434176007E0123054A834000200B
:102C900011680B431360E0BD0009084000F833FCE5
:102CA0001C0808404B790A79C97842EA0322437E1E
:102CB00001F00301DB0601D5FFF7C4BFFFF78EBFAC
:102CC000417E027ECB064FEA42124CBF084B094BB5
:102CD000890713441A6822F4001248BF42F0805258
:102CE0001A60437E6FF3C30343760020704700BF32
:102CF00000090840000B084001F07F01F0B5EFF338
:102D0000118400238025EFF3108372B685F31188B8
:102D100083F310888718FE7CC9B1062922D80123C5
:102D200003FA01F13140D1B10125AC460CFA05F3AB
:102D300019429E4610D026EA0E06E4B2FE7484F3D1
:102D400011881C236B4322B160331844F0BD314617
:102D5000E9E703F59273F8E70135072DE6D1E4B210
:102D600084F311880020F1E710B5C0B1B9B1EFF3D9
:102D7000118200238024EFF3108372B684F311884C
:102D800083F310884B7E097EC3F30013184401239C
:102D90008B40C17C0B43C374D3B283F3118810BD45
:102DA000024B1868C0F30D20704700BF08080840A8
:102DB000037C61F34103037400207047EFF311803B
:102DC00000238022EFF3108372B682F3118883F31D
:102DD0001088074A136839B123F002031360C3B2A5
:102DE00083F311880020704743F00203F6E700BF29
:102DF0000408084008B540F02000064B064A186059
:102E00001968890601D5013AFAD10320FDF757FC6C
:102E1000002008BD10000840400D0300102208B536
:102E2000064B1A60064A1968C90601D5013AFAD15B
:102E30000320FDF744FC002008BD00BF100008403F
:102E4000400D030038B5036904460D4643B1437E87
:102E5000DB0606D5007E8001FFF7CCFF23691BB996
:102E600038BDFFF7DBFFF9E729462046FFF77FFE75
:102E7000F4E710B5EFF3118400238022EFF3108301
:102E800072B682F3118883F310886FF06D01E4B29B
:102E9000FFF7D8FF84F31188002010BD084601F029
:102EA00003B910B5182001F007F9044618B118222B
:102EB000002101F0CFFC204610BDFFEC70B5EFF310
:102EC000118500238022EFF3108372B682F31188FC
:102ED00083F31088037CDA060ED50A4B1B68DB07E8
:102EE0000AD5094E0520346844F0010324F001049A
:102EF000336001F0B5F83460EDB285F3118800203D
:102F000070BD00BF0808084004080840064B074A87
:102F10001A6002F16042D2F8E83A02F6E82243F081
:102F200004431360704700BF100B0840180008608E
:102F3000F0B5057E204F6D01EB5903F00043002AE8
:102F400033D0C688541E3444B4FBF6F4467E134393
:102F500006F0030643EAC443012E184E08BF43EAB5
:102F60004473EB51457E047E05F003056401012D99
:102F7000A35907D1124D2D68ED0554BF43F080537E
:102F800043F0005323F08043033243F00443921094
:102F9000A351037E00201B0303F1804303F50123AB
:102FA000824201EB800402DCF0BD0124CEE72468FC
:102FB00001301C60F4E700BF100908400009084018
:102FC00008080840F8B50E6907460C465EB90B7E46
:102FD0002F495B015A5842F000625A50637E66F3F3
:102FE00082036376F8BDF3881BB94B7E43F0400340
:102FF0004B763289F588AA4208D3637E590605D4F8
:1030000020460021BDE8F840FFF7B1BD637EAD1A50
:103010006FF38613002D63760ADDE388AB4207DC8D
:1030200016D13379DB0703D5637E43F04003637623
:10303000217E184B4A01D258EB1C92B2B2EBA30F7F
:1030400008DA154A012310688B4003431360C9E76F
:103050001D46EDE733892A46316820461944FFF7BB
:1030600067FF637E43F004036376237E23B97B7C92
:10307000052262F307137B743289F3881544ADB2DD
:10308000AB423581AED8637E5A06ABD4B8E700BFF9
:1030900000090840180908403408084030B50346C4
:1030A0000B4C1A1D1B1A994200DC30BD2368C3F378
:1030B000072502F8043C02F8035CC3F30745C3F399
:1030C000076302F8025C02F8013C1346E9E700BF1F
:1030D00000100840002882B006DD002303490433B5
:1030E0000A6898420192FADC02B07047001008406A
:1030F00070B505460C4622695AB9237E1A485B0111
:10310000195841F000611950637E62F382036376BF
:1031100070BDD18819B92046FFF729FDEBE7E38898
:10312000124E5A1E1144227EB1FBF3F152014B4361
:10313000905943EAC1430C4900F060400343935166
:10314000237E5B015A5842F004425A50637E43F09A
:1031500004036376237E002BDAD16B7C062262F3B4
:1031600007136B74D4E700BF000B0840100B084036
:103170001A4B024670B5C0688B60EFF311850023CF
:103180008024EFF3108372B684F3118883F31088E0
:10319000537E13F008031DD114694B613CB9537E73
:1031A00013F00406C2E9041109D0204603E0506977
:1031B000416118465161EDB285F3118870BD13F07D
:1031C0001004114603D0FFF7FDFE3046F3E7FFF78A
:1031D0008FFFEAE76FF00F00EDE700BF000089FF07
:1031E000044B1A6842F400721A601A681207FCD580
:1031F000704700BF0408084038B5437E0446DB062C
:103200003AD5037E34495B015B581D0432D5EFF398
:10321000118500238022EFF3108372B682F31188A8
:1032200083F31088027E5201535823F4004343F085
:1032300090435350294A037E590102EB4313186807
:103240008007FCD58B5843F002038B50207E800111
:10325000FFF7D0FD2249207E01220B68824023EA3D
:1032600002030B606FF06D012046FFF7EBFDEDB23E
:1032700085F31188002038BDEFF3118500238022EB
:10328000EFF3108372B682F3118883F31088FFF78F
:10329000A7FF027E13490A205201535823F400432A
:1032A00043F090435350FDF70AFA237E0E4A022161
:1032B0005B010B489950A2F54172136843F4806397
:1032C0001360227E036802F1100101228A4023EA82
:1032D00002030360C6E700BF000908400809084070
:1032E0001C080840000B0840080B0840002210B5DD
:1032F000044611466030FFF71BFE637C042262F334
:1033000007136374BDE81040FFF700BE10B5044614
:10331000FFF766FF027E0A200A495201535843F024
:10332000804343F400135350FDF7C9F9064A0020C7
:10333000136843F480631360637E43F0080363768D
:1033400010BD00BF000B084004080840427E034641
:10335000D20601D4FFF7DABF027E064852011158A7
:1033600041F40011115000205A7E42F008025A76B2
:10337000704700BF0009084010B5EFF31184002327
:103380008022EFF3108372B682F3118883F31088E2
:1033900029B1FFF795FCE4B284F3118810BDFFF763
:1033A000D5FFF8E710B50269044622B9437E62F3FF
:1033B0008203437610BD0021FFF7D9FB637E6FF3D4
:1033C000820363765B07F5D421460248BDE81040CE
:1033D000FFF78EBEC80C0024344A00202DE9F047C8
:1033E0001368334C23F001031360FFF703FDE0681B
:1033F00018B103682146DB689847FE232D4FDFF89C
:10340000C48000264FF0FF0A4FF01C09E3742375B7
:1034100009FB06F53846C8F800A06FF06D01C8F842
:1034200000A20136FFF70EFD05F1780305F59C7546
:1034300007F1C40023446FF06D01254408F1200812
:103440005A781C3722F04C025A70FFF7FBFC6B795C
:10345000072E23F04C036B71DAD1174B4FF0FF327C
:10346000002114481A604FF001125A600B23134ACE
:10347000136042F8043C52F8143C23F4FE6342F813
:10348000143C4022238A23F4706323F00403238234
:1034900002232372FFF7D6FB402200210848FFF7E2
:1034A0009DFBBDE8F047FFF731BD00BF04080840B1
:1034B000C80C0024280D00241808084014080840EF
:1034C000EC0D0024080908402DE9F34700F592753A
:1034D00004466FF046012846FFF7B4FC04F1600093
:1034E0006FF046010190FFF7ADFC94F83D31667D29
:1034F0006FF3C303019816F0600F84F83D3194F820
:1035000079306FF3C30384F87930238A23F0010301
:103510004FEA03534FEA135343F44053238205D039
:1035200004F115012046FFF740FB44E0A37E94F828
:103530001CE094F817C0277E617EE27E4CEA0727E4
:1035400041EA032194F8169042EA0E220FFA87F816
:103550000BB20FFA82FEB9F10C0F28D80FF2040A51
:103560005AF829F09935000869360008AF35000887
:10357000C1360008AF35000863370008A5370008DA
:10358000A5370008AD370008CB3700082135000803
:1035900021350008B735000894F810C01CF0040F5E
:1035A00005D0022A03D116F0800F00D01FB3237C70
:1035B00043F001032374237CDB0716D594F878309D
:1035C000284692495B015A5842F400125A5094F826
:1035D000793043F0080384F87930FFF797FE237CB5
:1035E00043F001032374FFF791FC0023A4F85E303D
:1035F00002B0BDE8F08706F01F06012E31D0022E82
:103600000DD0002ED3D10029D1D1CCF30013CCF3AF
:10361000400CA1774CEA430C84F81DC015E003F080
:103620007F03062BC3D8C3EBC3030A064FF0020285
:103630004FEA83034CBF603303F5927323445B7EF0
:10364000C3F3C00363770023A37704F11D01FFF7E1
:103650006FFC637C042262F307136374FFF756FC6C
:10366000A9E76777A777F0E7207C10F0040F9ED0DA
:10367000002A9CD106F01F06022E16D1002F7FF4DF
:103680004FAF03F07F03062B3FF64AAFC3EBC303F4
:1036900098000B064CBF603000F592702044FFF795
:1036A0000FFB2046FFF722FE85E7002E7FF438AFA0
:1036B000012F7FF435AF034662F304132374F0E760
:1036C000207C10F0040F3FF472AF002A7FF46FAF3C
:1036D00006F01F06022E12D1002F3ED103F07F0309
:1036E000062B3AD8C3EBC3030E064FEA83004CBF48
:1036F000603000F592702044FFF728FED1E766BBEA
:10370000012F03D140F010002074CAE7022F24D10A
:1037100011F0FF0F21D1090AA37C0139042914D823
:10372000DFE801F0030B0D0F1100012262F3030328
:10373000A374237C43F02003C0E70222F6E70322B0
:10374000F4E70422F2E70522F0E76FF30303A37422
:10375000237C43F001032374EBE701077FF527AFD8
:10376000DEE6F2067FF423AF53EA0E037FF41FAFC9
:103770007F2F3FF61CAF637C03F00F03022B3FF457
:1037800016AF234A136823F4FE6343EA0C13136055
:10379000204B228A1340BCF1000F01D043F4827306
:1037A00023827EE7F3067FF402AFB9E6217C4F0760
:1037B0007FF5FDAEF0067FF4FAAE58EA03037FF41E
:1037C000F6AE012A7FF4F3AEAAE6227C51077FF51C
:1037D000EEAEF2067FF4EBAE53EA0E037FF4E7AEF3
:1037E00004F115012046FFF7E0F900287FF4E3AE6D
:1037F000228A18F0FF0F084B03EA020314BF43F4B8
:10380000027343F480732382D5E600BF00090840A9
:1038100000080840FBF0FFFFF7F0FFFF2DE9F74F2E
:103820008B498C4B0C681B688B4A03EA04001C40D4
:1038300002EA00020A6000F0A88025030ED5874B3B
:10384000874A1D68126815402D0C40F0A9801B683E
:10385000FF21844A1B0C002B40F09B8063030FD593
:103860007E4B7F4A1D6812681540ADB2002D40F0B6
:1038700009811B68FF217C4A9BB2002B40F0E2804B
:10388000002C10DA794A0121794D1368284623F07B
:1038900001031360FDF7D2F9E86820B102685269AC
:1038A0000AB12946904721050AD57149C86818B15F
:1038B00003681B6903B1984700216D48FDF7BEF905
:1038C000E2065CD56B4B1D6805F00F08B8F1060FDA
:1038D00055DC05F4F013B3F5002F00F07481B3F557
:1038E000402F00F07D81B3F5802F48D1C5F30A1534
:1038F000002D44D05E4B1C2606FB08369946D6F8B0
:103900003471002F40F04A8196F83CA1BAF1000FC3
:1039100040F04081D6F82C717B7C03F0F003102B33
:1039200040F03881402D2B4607F11D00A8BF4023F1
:103930001FFA83FB00935946FFF7B0FB009BE81A80
:10394000FFF7C8FB96F83D3102226AF3820386F83E
:103950003D317B7CA7F85EB062F307137B7403F004
:10396000F003202B02D13846FFF7AEFD1C2303FBEA
:10397000089898F83D316FF3820388F83D313E4B4B
:103980001C4200F04581FFF727FD002003B0BDE891
:10399000F08FD80701D5106811605B0820325AE714
:1039A0000026DFF8C080DFF8D8A0DFF8C4B0EF074A
:1039B00037D54FEA461959F80870DAF800301F4039
:1039C000F8071BD5012316F0FF0049F808309BF8D3
:1039D00011302BD103F0F003602B0FD12748FFF7F4
:1039E000E1FC9BF83D3113F0040107D1FFF78EFA9B
:1039F0009BF8113061F307138BF81130B90702D52A
:103A0000022349F808303A070BD59BF8113003F030
:103A1000F003202B02D15846FFF756FD082349F842
:103A200008306D0806F10106C1D117E703F00F0356
:103A3000022BE3D11C2303FB00B000F59270FFF7CB
:103A4000B1FCDBE7DF0700D511605B08203214E72B
:103A500014000840180008400AFCB0F81808084094
:103A60001C080840080B08400809084004080840E2
:103A7000C80C00242000084000108000EC0D002439
:103A8000140808404FF0600B4FF00008EE0773D5A4
:103A90006D4A4FEA481A6D4BDFF8C0911B681668F3
:103AA00001225AF8097002FA08F23242009218BF55
:103AB00043F080031F4017F0010301933CD0009BAB
:103AC0005FFA88FC1C2126EA03065F4B1E60012377
:103AD0004AF809305E4B01FB0C3118465A7C6031C4
:103AE000BCF1000F4FD102F0F002502A0ED1FFF7C7
:103AF00069FA574B93F8792012F0040106D1FFF7C9
:103B000005FA534B5A7C61F307125A74197C8806E4
:103B100012D5DFF84CC16FF345119A7CDCF8000038
:103B200002F00F0E6FF3030200F0700040EA0E1077
:103B3000CCF8000019749A743A0702D508234AF8A1
:103B40000930FB0607D5424800EB0B01FFF73AFAB4
:103B500010234AF8093038060ED5019B4BB9009B5B
:103B60003B4826EA0306384B00EB0B011E60FFF7CB
:103B700029FA80234AF809306D0808F101080BF191
:103B80001C0B83D17CE602F00F02022AD4D1FFF78E
:103B900019FAD1E72846FFF79DFAE7E63889FE884B
:103BA0003B68361A1844AE42A8BF2E461FFA86F864
:103BB0004146FFF773FAA81BFFF78CFA398988444E
:103BC000A7F80880DBE6224B5B7C03F0F003102BA8
:103BD0007FF4D5AE1F4A136843F080631360CEE6CE
:103BE0001B4D082105F11500FFF758FA95F915301E
:103BF000002B0ADB2A7FEB7E53EA022305D06B7C85
:103C0000012262F307136B74B9E66B7C0222F8E7BA
:103C1000A3047FF505AE104A1368A2F6F40223F45C
:103C2000FF6323F0070343F04003C2F8F438D2F8EF
:103C3000F83743F48073C2F8F837136823F47053ED
:103C400043F4C0531360EBE5340808401008084003
:103C5000C80C0024000B084000090840080908406F
:103C60000408084038B50B4CE060214603681B6827
:103C70009847054618B10023E360284638BD7520F3
:103C8000FCF75AFE01212046FFF798F80223237221
:103C9000F3E700BFC80C002470B50446EFF31185AC
:103CA00080260023EFF3108372B686F3118883F326
:103CB0001088FFF791FBEDB285F311880E4D204679
:103CC000236829465B689847EFF311840023EFF3DC
:103CD000108372B686F3118883F310887520E4B2DE
:103CE000FCF716FE00212846FFF768F80020E86080
:103CF00084F3118870BD00BFC80C002470B5284D36
:103D0000E86808B1FFF7C8FFEFF3118600238022AF
:103D1000EFF3108372B682F3118883F310880024C6
:103D200000211F48F6B2FFF749F875202C72FCF706
:103D3000EFFD214622467520FDF73CF8FF23194A86
:103D40004FF4806013602032C2F8E0311360C2F893
:103D5000003220321360C2F8003220321360C2F801
:103D6000003220321360C2F8003220321360C2F8F1
:103D7000003220321360C2F800324FF0FF320A4B9B
:103D80001C605C605C62DC609A60FFF733F8FFF7F0
:103D900045F86B7C64F303036B7486F3118870BD84
:103DA000C80C00240809084010080840F8B5944BD6
:103DB0001A6822F0007242F080721A601A6851018B
:103DC000FCD59048FEF79CF98F48FEF799F98F488B
:103DD000FEF796F98E4FFFF791FF8E4B4FF4F4727A
:103DE000002118463E4600F035FD8B490246034649
:103DF0004FF01C0E4FF0400C42F8601B0021426057
:103E0000FE228066C27402750246C0F82C010EFBC9
:103E100001041C325764106504F1780594F8794068
:103E200044F010046C70CCB2013182F85C4064F054
:103E30007F04072982F848406C786FF301046C70A6
:103E4000A2F84AC0E3D100221C274025D1B2C3F812
:103E50002461C3F830011C3383F8201183F80C115E
:103E600007FB0201013291F83D41072A6FF301047B
:103E700081F83D41A3F80E51E8D100226749752031
:103E8000FCF798FF002803DABDE8F840FFF736BFDB
:103E90008022634D634B644F1A602A683E46634C30
:103EA00042F040022A600320FCF709FC3B68002B2B
:103EB00001DB013CF7D1012333605C4B3268D20750
:103EC00001D5013BFAD103200024FCF7F8FB584B45
:103ED0004FF4803214201A6000F0C2F8554A3220A4
:103EE000136843F0C00313602B6823F0005343F0C2
:103EF00080432B6000F0B4F84F4B4FF480601C609F
:103F0000A3F5C0631A68A3F2DC7322F4C052C3F8AD
:103F1000DC27D3F8DC2742F00302C3F8DC2740F2A9
:103F200001221A6002F592025A604932C3F8E02079
:103F30004932C3F8E4204932C3F8E8204932C3F8D3
:103F4000EC204932C3F8F0204932C3F8F420FEF7E0
:103F500051FFFEF763FF394B4FF0FF32FF211C602A
:103F6000F03343F8EC4C43F8CC4C43F8E82C344A9B
:103F700043F8E44C186820330028B4BF4FF00840E1
:103F8000002043F8200C43F8104C43F8181C9342CF
:103F9000F0D12C4B0022FF202B491C682033002C31
:103FA000B4BF4FF00844002443F8204C43F8102CD1
:103FB00043F8180C8B42F0D1244925480A604FF091
:103FC000FF32244B1A600268234B22F07F4222F416
:103FD0007C0222F47C4222F0FF0213438122036020
:103FE0001E4B0C480B6000210E4B1A60FEF7E6FEDC
:103FF000FFF7F2F97520BDE8F840FCF79DBC00BF63
:104000000C4802580BAC08000CAC08000AAE0900C2
:10401000EC9E0008C80C0024D09E00081D38000843
:104020000C0008400800084010000840400D030044
:104030003800084000000840000E08401008084002
:10404000E0090840000B0840E00B08401800084059
:1040500014000840040008400AFCB0F810380C00B6
:1040600082B0002345F261610093009A824201D33D
:1040700002B070470193019A8A4203D9009A013233
:104080000092F2E7019A01320192F4E70A460146F2
:10409000034808B500F052F8024B186008BD00BF95
:1040A000089F0008B00E0024024B0146186800F07B
:1040B000C7B800BFB00E0024024B0146186800F0DC
:1040C0001BB900BFB00E0024024B0146186800F077
:1040D00071B900BFB00E0024F8B50D46044616466F
:1040E00000F05AF805F11F036168AA19082523F0AA
:1040F0000F03012622F00F02A3F11007D01B014489
:104100001038C4E9011743F8105CA1684E60A3F1B0
:10411000080143F8080CA2F108004D60E060204659
:1041200042F8085C53F8083CE2683343536000F0FF
:104130005FF82046BDE8F84000F052B801F10F03E7
:10414000A2F5A27223F00F0311444FF4A272184695
:1041500070B5CC1A00211D4603F5A27600F07AFB5B
:10416000034600F1200200F5A071A2F110009A614F
:1041700010321033D8618A42F7D1284600F007F890
:10418000284622463146FFF7A7FF284670BD012288
:10419000002100F09BB9FFEC104B37B51C680546B9
:1041A0004CB101A900F0ACF901980028D4BF00205F
:1041B000012003B030BD04F0F3FA00280CDB2846E0
:1041C00004F012FA002801DB0120F2E700F000F908
:1041D0000368002BF3DCF7E72046EAE7040300243A
:1041E000024B1B680BB904F04BBA70470403002460
:1041F00038B5054608680C4600F015F8421C05EB7A
:10420000001005EB0212836923B1196811B120680F
:10421000814205D39460C4E9023203B1DC6038BD49
:104220001A469B68F0E7B0F5800F07D2030900201B
:10423000012B00D8704701305B08F9E71220704766
:1042400070B505460C46A9B1FFF7A6FF98B9EFF384
:10425000118300228021EFF3108272B681F311885E
:1042600082F31088D5F84021DBB22260C5F84041C6
:1042700083F3118870BD54F8043CA4F1080123F0C5
:10428000010344F8043C54F8083CCA185068C607B7
:1042900013D4CB58D2E902061344B06008B1D668F3
:1042A000C660126854F8080C104444F8080C5A68A8
:1042B00002F0010202435A601A4654F8043CCB1A39
:1042C0005868C00710D4D3E90210816009B1D868DA
:1042D000C860196854F8080C08441860516801F067
:1042E00001010143516019462846FFF781FF284626
:1042F000BDE87040FFF774BFF8B506460F46EFF310
:10430000118300228021EFF3108272B681F31188AD
:1043100082F310880022D0F84041DBB2C0F840217F
:1043200083F31188002C3AD1002F36D007F11705FE
:1043300025F00F05AF4230D83046FFF72DFFB5F519
:10434000800F33D22846FFF76EFF06EB001084691A
:1043500004B32268A368AA422AD3E2689360A368E0
:104360000BB1E268DA602368581B0F280CD923448C
:10437000611960514D6025605A6802F001020243E4
:1043800030465A60FFF734FF6368083443F0010396
:1043900044F8043C3046FFF723FF2046F8BD25686B
:1043A000214630462C46FFF74BFFBBE71220CCE7F7
:1043B0001C46CDE713B50191FFF79EFF044618B1E7
:1043C000019A002100F046FA204602B010BDFFEC31
:1043D00008B500F0E7FA08B1143008BD0048FCE762
:1043E000B40E0024002303600B6813B90860486012
:1043F00070474B681860FAE70B6802468BB180B1D2
:10440000834208D11A680A604A689A4209D1002397
:104410004B6070472BB118461B689342FAD100F0ED
:104420000BB8704703682BB11A68026002B942608A
:1044300000221A60184670470A68036852B14BB1EF
:104440004A689A424FF0000215BF1968486001603F
:1044500002601A6018467047002303604B6843608F
:104460000A6812B90860486070471860FBE70023CB
:1044700043600B68036013B9C1E9000070475860DE
:1044800008607047D0E9003232B90B6033B94A6036
:104490000023C0E9003370471360F7E75A60F7E77D
:1044A00007B504460191009200F088FADDE900109A
:1044B000A047FCF7AFFB30B1B2F5004F03D212B208
:1044C0000280002070476FF01500704708B530B1CA
:1044D000B2F5004F03D212B20280002008BDFFF7F0
:1044E00077FF162303604FF0FF30F7E728B121B1C3
:1044F000038800201BB20B6070476FF015007047F7
:1045000010B5FFF7F3FF041E05DA6442FFF760FF02
:1045100004604FF0FF34204610BD1F299FBF0123C8
:1045200003FA01F103680B439ABF036000206FF0A8
:10453000150070471F299FBF012303FA01F103688B
:104540008B439ABF036000206FF015007047002373
:104550000360184670471F299DBF036823FA01F1C5
:1045600001F001006FF0150070470FB41FB506ABE6
:1045700053F8041B0191039303F0C2FF039A5030D8
:10458000019900F079F805B05DF804EB04B07047CC
:1045900070B5044630B300F0D8F80121201D002684
:1045A00000F022F8012104F1500000F01DF8012173
:1045B00004F19C0000F018F8D4F8E85025B9204622
:1045C00000F0CBF8304670BDB5F844309B0707D5F6
:1045D0000121284600F008F836EA200628BF0646E2
:1045E0002D68EBE70646EDE7F8B5436805460F464C
:1045F000002B3EDBB0F844309B073AD500F0C0F802
:104600006C69FCB1EE69B44207D1284600F0D7F8D6
:10461000EC696969641A2046F8BD2B6A9C4226D170
:10462000361B32462146686803F0A0FC00280DDAEC
:1046300095F8463043F0020385F84630FFF7C8FE90
:1046400004686442284600F0BAF8E4E70444361AE5
:104650000FB1002EE5DC6B692644EB61B442D4D087
:10466000EB695A1CEA6114F8012B1A70F6E7002472
:10467000E8E76FF00804CEE730B589B004460D4690
:10468000014603A8019200F0CBF8204600F078F82C
:104690002946019A03A800F0B3F90546204600F028
:1046A0008EF8284609B030BD08B5FDF767FA002836
:1046B00003DAFFF78DFE0068404208BD38B50122DD
:1046C000044600212C30FFF701FF4FF0FF35002397
:1046D00004F130006563C4E9453300F040F804F1AB
:1046E0007C00C4F8805000F03AF804F1C800C4F827
:1046F000CC50BDE8384000F032B838B504462C3014
:10470000FDF73CFA0023C4F81831D4F814516DB900
:1047100004F13800FFF7C8FF04F18400FFF7C4FF7D
:1047200004F1D000BDE83840FFF7BEBF284650F87E
:10473000083BC4F81431FDF721FA002801DAFFF72D
:1047400047FE2846FFF7B0FCDFE710B504462046D9
:1047500003F04AFF0028FADB10BD03F091BF08B553
:1047600000214FF0FF330122083001814360FFF741
:10477000ADFE002803DABDE80840FFF729BE08BDFA
:1047800070B5044604F048F80546E368984212D034
:1047900004F10806304603F027FF031E07DAFFF78F
:1047A00017FE0368042BF5D08C2BF3D05B422BB99A
:1047B0000123E56001E0238A0133238270BD10B537
:1047C000044604F029F8238A012B0ED1002304F1BA
:1047D000080023824FF0FF33E36003F051FF00280D
:1047E00005DABDE81040FFF7F3BD013B238210BDA1
:1047F00001210069FFF7F8BE38B504460D4621696E
:10480000284600F01FFE013003D0E3680133E36067
:1048100038BDFFF7DDFD0368042BF0D0F8E7FFECAF
:10482000094B03604B6963B1B1F84430074A13F494
:10483000807F074B18BF134683600023C0E9033114
:104840007047034BF8E700BFF9470008F14700083D
:1048500083540008002A43D010F0010F034639D0DA
:10486000013A03F8011B012A38D9F0B541EA0125C4
:104870009E07ADB22BD0023A23F8025B032A18D967
:104880005C0745EA054616BF141F144643F8046B3F
:10489000224603EB040C072A13D8E2086FF007073F
:1048A00007FB02423C40032A234484BF043A43F8F6
:1048B000046B012A02D9023A23F8025B02B1197093
:1048C000F0BDACEB0207083AC7E90066E3E7032A4C
:1048D000D6D8F0E7012AC8D8197001E0002AFBD128
:1048E0007047421E11F8013B02F8013F002BF9D13D
:1048F000704710B5044692B10A440B46184601337E
:10490000934203D100232370034609E013F8010CFE
:1049100004F8010B0028F1D1581A013810BD0B46DC
:1049200013F8012B002AFBD1F6E703461A460133A0
:1049300011780029FAD1101A704702440139034650
:1049400010B5934207D011F8014F03F8014B002C2A
:10495000F7D1934200D110BD03F8014BF9E7FFEC0A
:104960000E4B002230B5D3E900548C4209D1C56109
:10497000836823F4805323F00F03194381600020E0
:1049800030BDA94202D1C1612146F1E701320833AD
:104990001F2AE8D1C1614FF48051E9E7109F000858
:1049A000C06970471FB5002001A903F0C3FD0028AE
:1049B000ACBF0298002005B05DF804FB2DE9F04182
:1049C0000A4C226842B90A4D0A4E0B4FDFF82C8080
:1049D000B54203D101232360BDE8F08155F8043BC3
:1049E000BB42F5D34345F3D29847F1E7B80E002414
:1049F00088A2000888A200080000000888A2000819
:104A000007B5009200220B46114600F003F803B0F0
:104A10005DF804FB2DE9F04F8FB004460025DDF86A
:104A200060B093F800A0BAF1000F00F00784BAF16B
:104A3000250F08D0013302932368514620460135E3
:104A4000D94698472CE193F801A09A1CBAF1250F9A
:104A50000292F1D000270A223E46B846B8F13F0F35
:104A60004BD8BAF12B0F3DD014D8BAF1200F3BD060
:104A7000BAF1230F3ED0AAF13003DBB2092B4FD895
:104A800018F4807F12BF02FB073748F0800802FB52
:104A9000063607E0BAF12D0F29D0BAF1300FEAD16E
:104AA00048F00108029B13F801AB0293BAF1000F22
:104AB000D4D1AAF14503022B78D80AF1200A48F490
:104AC00000585FFA8AFA18F4807F08BF0627BAF107
:104AD000650FF9B240F08A80013148F48048C9B2CC
:104AE00000228BE048F0020848F00408DAE748F0BA
:104AF0000808D7E748F01008D4E7B8F5007FBAD324
:104B0000BAF17A0F2DD0BAF1740F2AD0BAF16A0F28
:104B100024D128F480681FFA88F848F42068C1E797
:104B2000BAF12A0F10D118F4807F5BF8043B02D051
:104B300023EAE377B6E7002BA7BF48F080081E46BC
:104B40005E4248F08808ADE7BAF12E0FD8D118F4CC
:104B5000807F40F0738348F48078A3E7BAF16C0F4C
:104B60000BD118F4007F18BF48F4006828F480685F
:104B70001FFA88F848F4007894E7BAF1680F0BD16F
:104B800018F4806F18BF48F4006828F400781FFA02
:104B900088F848F4806885E7BAF1700F02BF28F4FE
:104BA00020681FFA88F848F4007882E7AAF16503C4
:104BB000022B88D9BAF1630F00F0AD810AF0DF0350
:104BC000532B40F0D881D9469F4B59F804ABBAF12A
:104BD000000F08BF9A4618F4807F504614BF39462C
:104BE0004FF0FF3100F04FFC07469CE1BAF1660F31
:104BF0007FF476AF0A4648F400480F210BF107090D
:104C00000F2908A829F0070928BF0F21B9EC020BCA
:104C100000F046FB9DF8243003F00902012A42D03F
:104C200018F0020F42D118F0040F0CBF4FF0000A29
:104C30004FF0200A13F00C0F44D0BAF1000F14BF4C
:104C400004230323B3420CDA18F0080FA6EB030683
:104C500008D137462368202120469847013FF9D1E3
:104C600035440026BAF1000F04D02368514620468F
:104C7000013598479DF8243008F40058734F13F01D
:104C8000080F734B18BF1F46A5EB070A0AEB070571
:104C900017F8011B69B93746002F40F0C982354427
:104CA000CB46029BBDE64FF02D0AC3E74FF02B0A1F
:104CB000C0E7B8F1000F01D02039C9B223682046FF
:104CC0009847E3E7C3B2DDF820B00193614B019A46
:104CD00018EA030F1AD1134608A904330B440199AB
:104CE00019B113F80119302929D01BF1040F2BDB5E
:104CF000934529DABBF1000F48F4004802DB019B21
:104D00009B4524DA0BF10107019BDF1B0FFA88F3A7
:104D1000002B0393B6BF2BEAEB7305230133BAF1E3
:104D2000000F00D00133A7B17A1C1344B342B4BFC3
:104D3000F61A002618F0090F1BD1334614E001992A
:104D4000481EC1B20191CAE7019B5F1EDEE7002742
:104D5000DCE718F0100F18BF0133E7E720212046E9
:104D600004939047049B013B2268002BF6D1354405
:104D70001E46BAF1000F04D0236851462046013583
:104D8000984718F0080F0CD1B24604E00AF1FF3A38
:104D90003021204698472368BAF1000FF6D13544F8
:104DA0005646039B002B57DA2BEAEB739A46039384
:104DB0000EAB5B44133B0593ABEB0A03019A7942BC
:104DC00093423CBFCAF10003059A0AF1FF3A2CBF97
:104DD0003023D35C6A1C8A450492226824DA039942
:104DE000FF4303980139B842D8BF0F4618F0100F9F
:104DF00007D0791C05D12E21204601939047049DB0
:104E0000019BBB450AD19DF82520352A1AD805D12A
:104E10009DF8242012F0100F08BF31232268194694
:104E200020460135904736E7194620469047BAF1AB
:104E3000FF3F05D1AB1C2E212046049323689847E1
:104E4000049DB9E73123E9E710A0000808A0000895
:104E50000CA0000800C0FFFF9DF825102046312956
:104E60001EBF9DF8243023F010038DF824302368F2
:104E70009847002F23683DDD02354FF0010A2E21AF
:104E8000204698475745236823DA18F4005F2368C3
:104E9000204614BF452165219847BBF1000F04DB74
:104EA00032D19DF82430DB062ED5CBF1000B2D211D
:104EB0002368204698473021BBF1090F26DC236880
:104EC0002046984723680BF1300120460435984767
:104ED000E1E6019A2046013552458ABF0EAA3021EB
:104EE00052440AF1010A88BF12F8131C5FFA8AFAC9
:104EF0009847C7E718F0100F01D10135C5E72E21FB
:104F0000204602359847C0E72B21D1E70131ABF1AC
:104F10000A0BC9B2D0E7D94601270DF1200A59F88A
:104F2000043B8DF8203018F0080F15D1B04605E08D
:104F300008F1FF3823682021204698474745F7D3DA
:104F4000BE42A6EB070334BF00221A46C3F100039A
:104F500038BF002315441E440AEB0708C24501D19F
:104F60003D4498E6236820461AF8011B9847002E16
:104F7000F4D0013EF2E7BAF1640F08F4206302D0E6
:104F8000BAF1690F77D1B3F5206F61D10BF1070941
:104F900029F00709F9E80201002828F4805B71F183
:104FA00000032BF0100B06DA40424BF4805B61EB00
:104FB00041011FFA8BFB1BF4807F04D01FB950EA1C
:104FC000010300F0C3800DF120080A23424600F0DF
:104FD00039F9A0EB08085FFA88F81BF4807FCDF858
:104FE000048000F0B5802BF0010AB8451FFA8AFA58
:104FF00080F2B18044F21002FBB20BEA0202102AE6
:1050000003D12BF0110A1FFA8AFA1AF0100F00F0E0
:10501000AC800EAA424412F8192C302A40F09D8030
:105020002AF4C04A2AF0100A1FFA8AFA1AF0080F66
:1050300040F0AC801AF0010F05D0B34280F2C58079
:10504000F71AF3B24744A3EB050B5FFA8BFB98E02A
:10505000D94618F4007F59F8043B18464FEAE3712B
:105060009AD118F4806F97D018F4006F0CBF18B263
:1050700058B2C11790E7B3F5206F1AD10BF10709A9
:1050800029F00709F9E8020128F0060BBAF1580FD8
:105090001FFA8BFB46D0AAF16F03DAB2092A49D86E
:1050A000092B47D8DFE803F0502646464646174608
:1050B000463718F4007F0BF10409DBF8000001D03B
:1050C0000021E1E718F4806FFAD018F4006F0CBFEC
:1050D00080B2C0B2F4E728F0160B0A231FFA8BFB4C
:1050E0001BF4807F03D017B950EA01022ED00DF1D6
:1050F00020086BE7029B1B78562B0AD1029B0133D9
:10510000029343681A68079201682046FFF778FC0B
:10511000C6E54BF0100B1BF0100F01D04BF4804B89
:105120001023DDE718F0100F01D04BF4C04B4FF403
:105130000473D5E723682046252102359847236864
:10514000514620469847ABE50823C9E7B84644E7EF
:105150004346DA4659E7434657E71AF4804F01D1F0
:10516000013300E00233DBB260E741F206021AEAE3
:10517000020F3FF45BAFF3E723682021204601359F
:1051800098470BEB0503DBB2B342F5DBB342B4BF88
:10519000F61A00261AF0100F24D02368302120467A
:1051A00098471AF4804F12D10135BA46D0452BDB0F
:1051B000A7EB0800B845C8BF00200544B8F1000FB0
:1051C00029D1019B2B441D4665E547463BE71AF470
:1051D000005F05F10205236814BF5821782120469D
:1051E0009847E2E741F206031AEA030FDDD01AF00E
:1051F000020F05F10105236814BF2B2120211AF4A9
:10520000805F18BF2D21EAE72368302120460AF18C
:10521000FF3A9847CAE708F1FF330EAA204652FA30
:1052200083F25FFA83F8236812F8181C9847C5E7E1
:10523000236820212046013F98472DE528460FB0DE
:10524000BDE8F08F2DE9F84F13F400790746884642
:1052500016461CBF23F400734FF001091C46DD17EE
:105260003846414622462B4603F0F8FE092ABA4644
:10527000C3460746884609DC3032AB4506F8012BA9
:1052800008BFA245ECD23046BDE8F88FB9F1000F57
:1052900001D03732F1E75732EFE7FFECC2925D7D84
:1052A0002DE9F74F10EE904A07460E4614F00044E1
:1052B0001CBFB1EE400B0124B5EE400BF1EE10FA2D
:1052C00016D16FF00401431D44F00204091A302086
:1052D000CA18964209DC0025BB19002230465A71D3
:1052E0003C713D6003B0BDE8F08F03F8010BEFE7C0
:1052F000B4EE400BF1EE10FA02D744F00804EAE7EE
:10530000B0EEC07B9FED446BB4EE467BF1EE10FA3D
:1053100002DD44F00404DEE79FED417BB4EEC70BF1
:10532000F1EE10FA5DD5424908230F2501209FEDCB
:105330003E6B91ED107B20EE077BB4EEC67BF1EE69
:1053400010FA05D500FA03FCB0EE470BA5EB0C05EF
:10535000013B0839B3F1FF3FEBD132B125EAE573E8
:1053600001331A449642A8BF1646324B03EBC603DC
:1053700093ED007B30EE070B9FED2B7BB4EEC70B5C
:10538000F1EE10FA04DBB2EE047B013580EE070B80
:1053900007F10508DFF8A4A0DFF8A4B051EC100B6A
:1053A00003F076FE6FF0040389460090DB1B019347
:1053B000019B43449E428FDD52465B46009849461E
:1053C00003F04CFE00F1300C5946504600929946CD
:1053D0000A22002308F801CB03F040FE82468B46E8
:1053E000E6E7154908230F25012091ED106B20EE0B
:1053F000066BB4EEC76BF1EE10FA04DB00FA03FCA7
:10540000B0EE460B6544013B0839B3F1FF3FECD1E8
:10541000A3E700BFAFF30080FFFFFFFFFFFFEF7FB9
:1054200000003426F56B0C430080E03779C341431C
:10543000E0A0000818A0000898A000080080C6A4FA
:105440007E8D030037B50A468DF8070004460D46E9
:105450000DF10700012100F023F8002804DC4FF0D3
:10546000FF34204603B030BD0A2CFAD195F84630FF
:105470005B07F6D501212846FFF7B6F80028F0DAD9
:10548000EDE7002070470246014410B58A421346FA
:1054900001D1181A10BD1C780132002CF6D1F8E7A2
:1054A0002DE9F84380460F46164642B9FEF790FFB5
:1054B0004FF0FF34092303602046BDE8F883B2F8BB
:1054C00044309B0706D4FEF783FF092303604FF0A7
:1054D000FF3418E053693BB90A460146706802F090
:1054E00045FD041EE8DAF2E71046FFF749F93046B9
:1054F00000F04EF800280DDA4FF0FF343046FFF789
:105500005EF9002CD8DA96F8463043F0020386F8AC
:105510004630D1E7D6E906502D1A202D01D11F2F94
:105520001CD8BD42414628BF3D462A46A7EB050987
:10553000FBF75EFAF369B26908EB05042B4493426A
:10554000F36104D2B9F11F0F14D94F4607E00021CF
:105550003046FFF749F80028F4DACDE744463A46EA
:105560002146706802F002FD0028C5DB0444A4EB6C
:105570000804C3E7B9F1000FF9D021464A46F069A3
:1055800008EB0704FBF734FAF3694B44F361EEE7E9
:1055900010B5044630B9FEF71BFF092303604FF036
:1055A000FF3010BD4369F3B1FFF7EAF8206A626982
:1055B000904213D0E36994F847101B1A2046C4E9BF
:1055C00007220022591A84F84720012200F00DF822
:1055D000002803DA2046FFF7F2F8E0E72046FFF75D
:1055E000EEF80020DDE71846DBE700F000B870B504
:1055F00004460D461646FFF7CBFF002802DA4FF0AF
:10560000FF3070BD204600F010F80028F7DB0023C3
:1056100032462946606884F8473002F088FB013042
:105620004FF0FF3018BF0020EBE7426932B1B0F80D
:1056300044309B0702D50121FEF7D6BF00207047FA
:10564000022901D100F008BB7047FFEC08B5094BF7
:105650001B7813F0FD0F02D04FF0FF3008BDC307D9
:10566000FAD500F02FFB0028F6DB034B02221A705C
:10567000F4E700BFBD0E0024C413002410B5084C8D
:10568000606003F089FEFFF7E1FF002804DB054AB4
:1056900013680133136010BD6368002BF1D1FAE782
:1056A000C8130024C00E002408B5FFF7E7FFA0F1DF
:1056B00020035842584108BD034B1B78022B01D1EF
:1056C00000F026BB704700BFBD0E002410B5124C81
:1056D000236801331ED0114B1A68053B9A4219D931
:1056E0000F4B9B6803F1006303F500339A4211D21C
:1056F00003F0ACFE03F07AFE00F0D8FA03F084FE6B
:1057000003F04CFE204603F0BBFE2046BDE81040EF
:1057100003F060BF10BD00BF0000020804000208D3
:10572000AC0000240C4A002310B5144652F8231094
:1057300021B152F82310013942F823100133042B10
:10574000F4D1064B1B7833B9A36823B9022003F0C8
:105750002FFF3223A36010BDC8130024BC0E002409
:10576000024BD860DA68002AFCD17047C8130024C5
:105770002DE9F04FDFF810838DB00025BA4E0746B3
:10578000DFF808A388F800500495B46803F01AFE07
:10579000CDF80480B0460FB1CAF80070B34B4FF09B
:1057A000FF36CAF8085099461D70012003F0F6FE36
:1057B00027B1DAF80030002B00F02B820020FFF731
:1057C0005DFF0590059B002BF2DB012003F0DCFE62
:1057D000059B213B102BE8D801A252F823F000BF13
:1057E000255800083B580008A3580008AB5700088C
:1057F000AB570008AB57000837590008AB570008F3
:10580000D5590008915A0008DB5A0008375B000898
:10581000855B0008575B0008AB570008EF5B00088A
:10582000FB5800080220FFF73FFF002800F003822A
:10583000049B43F0010304935FE04FF47A70FFF799
:105840001DFF051EC0F2F7810220FFF72DFF002883
:1058500000F0F181681E042800F2ED81DFE800F01D
:10586000030B0E11140004218148FFF725FF049B50
:1058700043F00203DFE704217B48F6E704217D487B
:10588000F3E704217C48F0E71C252846043503F0A3
:1058900017FE0421079007A8FFF70EFF2C2DF4D167
:1058A000E5E70220FFF700FF002800F0C481049B19
:1058B00003F00303032B40F0BE81012300250220E7
:1058C00089F8003003F060FE03F0CBFD284603F0BA
:1058D000DDFD044610BB022089F8000003F05EFEE7
:1058E000D8F80830A3421ED8049B002443F00403D8
:1058F00089F800400493CAF80840019B1B781BB943
:105900005E4B019A1B78137041F21203022107A823
:105910000027ADF81C30FFF7CFFE46E728460135DB
:1059200003F0BAFDD2E7204603F0CAFD013040F093
:1059300055810434D4E73220FFF7A0FE051EC0F2E3
:105940007A8115F0030240F076812B19D8F80810FF
:105950008B4200F27081B5F5807F00F26C81DFF838
:1059600020B15946AA4214D1C820FFF79DFE002855
:1059700000F0618124B9424B4FF0FF321E681A607B
:1059800025F003052544AC4215D1049B43F00803E0
:1059900051E74FF47A70CDE90221FFF76FFE0590D1
:1059A00005980028C0F2478105980399029A01F8EA
:1059B000010B0132D6E7DBF80010204603F07AFD38
:1059C000204603F07DFD5BF8042B904240F00681F9
:1059D0000434D8E70220FFF767FE002800F02B818F
:1059E00000252F462EE0002D39D1711C37D00796A7
:1059F000244A5168C1B994460B46082003F0010EB1
:105A00005B08BEF1000F07D083F06D4383F43803C9
:105A100083F4034383F020030138EFD101314CF8C4
:105A2000043BB1F5807FE7D107A8002110F8013BC6
:105A300001317B400429DBB252F8233083EA172777
:105A4000F4D10435D8F80830AB42CCD8042107A8EB
:105A50000797FFF731FE049B43F01003EBE628465F
:105A600003F02EFD0790C3E7AC000024BC0E002419
:105A700028A10008B0000024B4000024C4130024AE
:105A8000C4120024C40E0024BD0E0024C813002438
:105A900007AB4FF0000B1D4664200293FFF7EEFDAD
:105AA0000028C0F2C8800BF1010B029BBBF1040F70
:105AB00003F8010BF0D1079B02200293FFF7F4FDDE
:105AC000002800F0B880029B184603F003FD5946F9
:105AD00007902846FFF7F0FD0FE707AB4FF0000BEC
:105AE0001D4664200293FFF7C9FD0028C0F2A38081
:105AF0000BF1010B029BBBF1040F03F8010BF0D17A
:105B0000079B02200293FFF7CFFD002800F093804F
:105B1000029B9A0740F08F80082B00F28C80184679
:105B200003F02CFD594607902846FFF7C5FD049B5E
:105B300043F040037FE60220FFF7B6FD00287AD04D
:105B400003F0CAFC0421079007A8FFF7B5FD049BEA
:105B500043F080036FE60220FFF7A6FD00286AD01D
:105B600007A9142003F0BEFC05460421069006A8F0
:105B7000FFF7A2FD294607A8FFF79EFD049B43F40B
:105B8000807358E66420FFF779FD002853DBC5B227
:105B90001E2D50D80220FFF787FD00284BD04FF470
:105BA000D07003F08DFC83464FF4D27003F088FC74
:105BB000264B9B453FD1264B98423CD1DFF894B011
:105BC0004FF4D07045EA0B0B594603F073FC4FF4C9
:105BD000D07003F075FC58453FF48FAE41F21213BC
:105BE000022107A8ADF81C30FFF766FDDDE54FF494
:105BF0007A70FFF759FDF0B1731C0DD141F2120319
:105C000007A80221ADF81C30FFF756FD6420FFF70E
:105C1000A7FD0DB0BDE8F08F049B03F01B031B2B09
:105C200009D13146002003F045FC002003F048FC78
:105C30008642E3D0D2E741F21233022107A8ADF841
:105C40001C30FFF739FD00230493AEE5FFECC29250
:105C50005D7D05C500ECC29238B50F4B0F4C002896
:105C600008BF184603F050F90D49206003F05CF9B5
:105C70000C4B00B118604FF0FF320B4D43211868F8
:105C80002A6002F004F9002805DB28602068BDE8DE
:105C90003840FEF709BA38BD149E0008DC13002412
:105CA0002CA10008D81300247800002410B5044C5F
:105CB000206801F0C4FE4FF0FF33236010BD00BF29
:105CC0007800002413B50F4C2368002B0FDA0E4B1D
:105CD0004321186802F0DBF8002803DA4FF0FF30A8
:105CE00002B010BD094B20601868FEF7DDF90122F3
:105CF0000DF10701206802F004F90128EED19DF8AA
:105D00000700EDE778000024D8130024DC130024FA
:105D1000024B0A460146186802F028B978000024B0
:105D200003464FF604720846934210B513D04FF65F
:105D30000C72934212D04FF60172934226D1FAF7B9
:105D40006FFF002804461FDA6442FEF741FB04603F
:105D50004FF0FF3418E003F019FDF2E70B78012B48
:105D600005D14C78012C05D0022C08D064B16FF01D
:105D70001504E9E74968807801F076FBE1E74B68B4
:105D80000024186801F0F6FB204610BD6FF01804DF
:105D9000DAE708B500F080FDBDE8084000F012B871
:105DA000002070471046704708B54AB14B688A68B2
:105DB00003F0050313438B6013B1086902F022FC62
:105DC000002008BD00234FF4DB720249024802F0B4
:105DD00068BA00BF38A100082EA1000813B5044618
:105DE000A36B20460191DB6A984701990028F7D000
:105DF000A36B20465B6A02B0BDE8104018472DE94E
:105E0000F74F458C0446B0F9263088462DB24FF046
:105E1000800B01920135AB42D8BF0025A38C1BB289
:105E2000AB420AD0638C2DB2A26A00201BB202F8EA
:105E30000380658403B0BDE8F08F019B002B30D058
:105E4000EFF3118AEFF3108772B68BF3118887F3A3
:105E50001088A38C1BB2AB421ED1E27802F0FF097E
:105E6000E2B90121A26B20466170926A904704F169
:105E70001A0002F081FBA26B06464946926A204650
:105E800090475FFA8AFA8AF31188E37863B9002EA3
:105E9000C4DA6FF00300CDE70026F2E76FF07F066B
:105EA000EFE76FF00A00C5E76FF07F00C2E72DE96A
:105EB000F74F836880460E4601925C6904F12C0915
:105EC000484602F059FB051E1FDB00254FF0010B71
:105ED000019B9D4204D2E378DBB10DB96FF07F05E1
:105EE000A36B012120469B699847E28D238E12B255
:105EF0001BB29A4206D1A36B1B6A1BB1002220463B
:105F000011469847484602F07DFB284603B0BDE89D
:105F1000F08F238EE28D19B212B28A421ED0626BCC
:105F20000133525C1BB2B4F932109942D8BF00233E
:105F30002386E36813F4E07F05D00A2A07D113F023
:105F4000400F18BF0D22013506F8012BC0E70D2ABE
:105F5000F9D113F4807F18BF0A22F4E7002DBFD1D6
:105F6000D8F80830002B4BD0D8F8005015F0400579
:105F700049D1EFF3118A8023EFF3108772B683F3D0
:105F8000118887F31088A26B294620465FFA8AFAA7
:105F900092699047E18D228E09B212B2914227D1C7
:105FA000A26B0121204692699047E18D228E09B2B1
:105FB00012B2914202D08AF3118889E7E278A2B93D
:105FC00004F11C0084F802B002F0D6FA8AF31188BA
:105FD000002803DBE378002B3FF47AAFE378002B53
:105FE0007FF47CAF6FF003057AE76FF07F00EDE799
:105FF0008AF31188A36B012120469B69984767E7C4
:106000006FF050056CE76FF00A0569E72DE9F04184
:1060100083685E6906F11805284602F0ADFA041E91
:1060200023DBF378002B36D13378013313F0FF07ED
:1060300034D0012F2DD1EFF3118800238022EFF30C
:10604000108372B682F3118883F3108833795FFA74
:1060500088F86BB9B36B30461B689847041E07DAA3
:1060600088F31188284602F0CDFA2046BDE8F08179
:10607000B36B30469B689847041EB36B03DA5B68CA
:1060800030469847ECE79B6901213046984788F3F2
:1060900011883770E6E76FF07F04E3E76FF01704CD
:1060A000E0E7F7B50E4600F1400700F1500557F85C
:1060B000044B8CB16368A26843F018033340134368
:1060C000A3604BB101A92069FEF710FA019B002BD8
:1060D00002DC206902F096FAAF42E8D103B0F0BDCD
:1060E0002DE9F84383680E4615465C6904F11E08E5
:1060F000404602F041FA071E4EDB002D4FD004F15E
:106100004002002352F8045B002D34D1103304F117
:10611000200944F8236004EB83034846736102F0CE
:106120005BFA638CB4F926201BB201339A42D8BFC4
:106130000023A28C12B29A4225D1484604F12C09C0
:1061400002F060FA484602F047FAE28D238E484694
:1061500012B21BB29A421EBF736803F001031D43C3
:1061600002F050FAE37893B145F01805294620462D
:10617000FFF797FF0DE00133042BC3D100236FF02D
:106180000F07736105E0756805F00405D5E7002D7C
:10619000ECD1404602F036FA3846BDE8F883736920
:1061A000002BF6D01D607561F3E7FFEC2DE9F04799
:1061B000836880460F4616465D69464B1B6823B1CF
:1061C000EB78ABB16FF07F0425E002F0A1F9002875
:1061D000F6D105F1200A504602F0CEF9041E1ADB72
:1061E000EB7803F0FF018BB3504602F00BFAE9E7BE
:1061F000EFF3118400238022EFF3108372B682F351
:10620000118883F3108807EB0608B84506D1E4B27D
:1062100084F3118834462046BDE8F0872B6917F8CF
:10622000011BD80703D50D2905D11A0705D4284627
:10623000FFF7D4FDE9E70A29F9D113F0240F03D0C1
:106240000D212846FFF7CAFD0A21F0E7D8F8002003
:10625000B146AB6B284682F040089B6AC8F38018B1
:106260009847B9F1000F01D1344623E02B6917F8A4
:10627000011BD80703D50D290AD11A070AD44246B3
:106280002846FFF7BCFD041E10DB09F1FF39E8E7E3
:106290000A29F4D113F0240F01D10A21EFE7424675
:1062A0000D212846FFF7ABFD041EF6DAB14501D2F9
:1062B000A6EB09046A8CAB8C12B21BB29A4204D0D2
:1062C000AB6B012128469B6A9847504602F09AF929
:1062D000A1E700BF040300242DE9F04700F12008E6
:1062E00004460E46404602F047F9051E1DDBEFF35B
:1062F000118700238022EFF3108372B682F3118896
:1063000083F31088E37803F0FF0553B3638C6FF0D9
:106310007F05A384FFB287F311881E4B002D1F68F1
:1063200099462CDA404602F06DF92846BDE8F08720
:10633000A36B0121204684F801A09B6A9847484638
:1063400002F01AF9A36B054600219B6A2046984784
:10635000002DDFDB628CA38C12B21BB29A42E7D114
:10636000D8E74FF0010A04F11A09F3E74FF47A7005
:1063700002F0DCF9D9F80030DB1BB34206D2A36B84
:1063800020461B6B98470028F0D0CBE76FF07305D1
:10639000CBE700BFE41300244FF0FF332DE9F041B9
:1063A0008B6005460B790C462BB14B6943F001031A
:1063B0004B6105230B610122002104F1200004F14F
:1063C0001A07FEF778F80122002104F12C00FEF7ED
:1063D00072F80122002104F11800FEF76CF8002287
:1063E000384604F11C061146FEF765F800223046D7
:1063F0001146FEF760F80122002104F11E00FEF7AD
:106400005AF80021384602F0E3FC0021304602F041
:10641000DFFC234628464FF4DB720249BDE8F04119
:1064200001F03FBF58A1000810B504460121FFF755
:1064300038FEA3783BB1002304F11C00A370BDE833
:10644000104002F0DFB810BD10B504460421FFF77C
:1064500028FE63783BB1002304F11A006370BDE8A5
:10646000104002F0CFB810BD70B583680E461546D7
:106470005C69A36B1B69F3B9B6F58D7F0DDAB6F5D0
:106480008A7FC0F2BC80A6F58A73052B00F2B78024
:10649000DFE803F0799BB5B5A2ACB6F5427F36D004
:1064A00040F209339E424ED040F207339E420AD05A
:1064B0006FF018008FE0984710F1190FDCD000281A
:1064C00000F09F8087E0EFF3118100238022EFF33B
:1064D000108372B682F3118883F31088228EE38DC5
:1064E00012B21BB29A420ADCE38D228E1BB212B2A8
:1064F0009B1ACAB282F311882B6000206BE0228EB7
:10650000E08D12B2B4F9323000B2121AF0E7EFF3B4
:10651000118100238022EFF3108372B682F3118879
:1065200083F31088A28C638C12B21BB29A4203DCF4
:10653000638CA28C1BB2DAE7A28C608C12B2B4F925
:10654000263000B2E1E7EFF3118100238022EFF360
:10655000108372B682F3118883F31088628CA38C47
:1065600012B21BB29A4206DAA38C628C1BB212B230
:106570009B1A013BBDE7628CA08C12B2B4F92630A5
:1065800000B2121AF4E7EFF3118600238022EFF332
:10659000108372B682F3118883F3108835F00202FB
:1065A00007D1E38D2386A36B1B6A13B111462046E6
:1065B0009847013D012D04D8638C2046A384FFF742
:1065C00043FFF6B286F3118897E742F21071204636
:1065D000FFF782FE70B970BD002D02DA6FF0150072
:1065E000F9E7A368002BF9DAA56086E74FF0FF33DF
:1065F000A36082E710F1190F3FF45AAFEBE76FF099
:10660000180040F201139E420BD0B6F5817FE2D113
:10661000002DE3D02B68E3606B682361EB68636156
:106620006BE7002DDAD0E3682B6023696B60636948
:10663000EB6062E770B504460D46EFF31186002368
:106640008022EFF3108372B682F3118883F31088EF
:1066500081F00103C37089B91821FFF722FD637827
:1066600023B104F11A00657001F0CCFFA3782BB1BF
:10667000002304F11C00A37001F0C4FFF6B286F3FE
:10668000118870BD10B5044600211A3002F005F8DB
:10669000002104F11C0002F000F8012104F12000A7
:1066A00001F0FBFF012104F12C0001F0F6FF04F1E1
:1066B0001E000121BDE8104001F0EFBF70B58368F6
:1066C00005465C6904F11806304601F085FF237821
:1066D000012B06D9013B2370304601F093FF0020C7
:1066E00070BD0021A36B204621709B6998472B68E1
:1066F0005B0604D44FF47A612046FFF7EDFDEFF31B
:10670000118500238022EFF3108372B682F3118883
:1067100083F31088A36B2046DB68984723791BB965
:10672000A36B20465B689847EDB285F3118820463D
:10673000FFF77AFE2046FFF7A5FFCDE710B54369C6
:1067400013F0010302D00023934201D1002010BDB9
:106750008468002C04DDCC5C032C03D01A2C03D0FD
:106760000133F1E70A20F2E70720F0E7F8B500254A
:1067700004462F46628CAEB2A38C12B21BB29A4270
:1067800010D1628CA38C12B21BB29A4204D1A36BBB
:10679000002120469B6A9847EEB12046BDE8F840AC
:1067A000FFF752BEA36B2046DB6A98470028E8D06B
:1067B000A38C2046A16A1BB2A26BC95C526A9047A7
:1067C000A38CB4F9262001331BB29A42A38400DCC7
:1067D000A7840135CEE7F8BD2DE9F341C58D00272B
:1067E000B0F9323004462DB2B8460135AB42D8BFBD
:1067F0000025A36B2046DB69984700282FD0268E02
:1068000036B2AE4220D0A36B01A920465B699847FF
:1068100001228DF803000DF103012046FFF78EFFE2
:10682000AE428046E5D0E38D01379DF803101BB2E0
:10683000626BBFB2D1542BB20135E385B4F932306B
:10684000AB42D8BF0025D4E7A36B1B6A002BDAD07C
:106850000122B4F93210204698470028D3D017B14E
:106860002046FFF7E1FDB8F1000F06D04146A068D1
:1068700001F03AFF2046FFF705FF02B0BDE8F081C6
:1068800008B5044B186818B103689B6803B19847B2
:10689000002008BD800000240020704700230B81E9
:1068A000406F4968C388CB8003681B6918477047ED
:1068B000C36B93F85430002B0CBF6FF07F000020A7
:1068C0007047704700207047C36B93F8550003284A
:1068D00094BF00200120704770B5036806460D463E
:1068E0009B689847044660B1C5802846FDF7E4FBE5
:1068F0000546206028B9336821462C463046DB68BF
:106900009847204670BD806890F8543013B101213B
:10691000FFF790BE704700218068FFF78BBEF8B587
:106920000446EFF3118500238022EFF3108372B643
:1069300082F3118883F31088C66E8C30FDF772FDE8
:1069400048B394F85530A1220227013B84F8553012
:1069500041680B681A7020229F715A7000229A7049
:10696000DA701A715A71DA7194F859705A721F728A
:106970000A2308613046CB8001230B7133681B6901
:10698000984794F85930EDB203F0030384F8593076
:1069900085F31188F8BD6FF00B00F2E72DE9F047A1
:1069A0000446EFF3118700238022EFF3108372B6C1
:1069B00082F3118883F3108800F17C084046FBF7CE
:1069C000D1FA94F85D30002B65D094F85B50002D1F
:1069D00061D104F19409D4F89460002E4CD072680F
:1069E000002133891068B2F808A01844B4F93220A5
:1069F000AAEB030AE38D01331FFA8AFA9BB2934292
:106A0000A8BF0023228E8DB212B293422BD1238EC7
:106A10001BB2934206D1B4F932100122204601394B
:106A200000F06BF815B12046FFF7FEFCAA451ED812
:106A30004846FDF7F7FC31462046FFF72FFF054695
:106A4000C9E7E58D10F801C00131626B2DB202F883
:106A500005C01AB20133E2859BB2B4F932209342E9
:106A6000A8BF0023CEE7AA45EBD81A46CFE7338963
:106A70001D4435816FF01B05D4F894302BB12346AB
:106A8000064AC821404601F0D5FEFFB287F31188BF
:106A90002846BDE8F0876FF00F05EDE7F76A0008BC
:106AA00038B584680869EFF3118500238022EFF37D
:106AB000108372B682F3118883F31088B1F90A301B
:106AC00013F16E0F0CD08BB9038104F19401FDF723
:106AD00089FC2046FFF762FFEDB285F3118838BDCF
:106AE00094F85630013B84F85630F5E701462046CD
:106AF000FFF7D4FEF0E7FFF751BF38B5C46B94F849
:106B0000593094F85A1003F0020584F85C20F1B172
:106B10007AB145B123F00203204643F0010384F823
:106B20005930FFF7FCFE012384F85B3094F85B00DA
:106B300038BD84F85B2035B943F00303204684F860
:106B40005930FFF7ECFE2046FFF728FFEEE7002D57
:106B5000ECD143F00303204684F85930FFF7DFFE01
:106B600084F85B50E2E710B5C06BEFF311840023AB
:106B70008022EFF3108372B682F3118883F31088BA
:106B800059B190F85D3013B9012380F85D30FFF7FB
:106B900005FFE4B284F3118810BD80F85D10F8E7BA
:106BA0002DE9F04F044685B0EFF311838026029360
:106BB0000023EFF3108372B686F3118883F31088F5
:106BC000D0F870904FF0000B0396B9F80630602BA8
:106BD00038BF60230193D4F88C80B8F1000F2AD01D
:106BE000D8F804603068EFF3118A039BEFF3108547
:106BF00072B683F3118885F310880021B4F822C09F
:106C00008FB2A28C0FFA8CFC12B294451BD1618C0E
:106C1000A28C09B212B2914204D1A26B002120468B
:106C2000926A904717B12046FFF70EFC5FFA8AFA86
:106C30008AF31188DFB900209DF8083083F31188AA
:106C400005B0BDE8F08F019BBB42E0D9A78CA26ADA
:106C50003FB2D25D4254A28CB4F92670013212B216
:106C60009742A28401DCA4F824B00131C6E704F104
:106C70008C00FDF7D7FB94F8552031464846013A81
:106C800084F855200122F780C6F810803271D9F8B7
:106C900000201269904700289DD0CDE770B50D46C1
:106CA00084680869EFF3118600238022EFF31083D4
:106CB00072B682F3118883F3108804F18C01F6B266
:106CC000FDF790FB94F85530013384F8553086F386
:106CD0001188B5F90A3023B92046BDE87040FFF7A6
:106CE0005FBF70BD41B1C06B428C838C12B21BB2CE
:106CF0009A4201D0FFF754BF704738B583685C698A
:106D000040F20933994200F0EA8012DC40F2073386
:106D1000994200F0A680B1F5427F00F0C48040F2B5
:106D2000011399422CD0B1F5817F58D06FF018052E
:106D30007BE06FF4506001440329F7D80329F5D8AC
:106D4000DFE801F002051017A26600256DE0002AB9
:106D500000F0E58054F85E3F1360A3889380A37928
:106D60009371F2E7002A00F0DA8094F8583013604B
:106D7000EBE7204684F85920BDE83840FFF7CFBD47
:106D8000002A00F0CC80E3681360236953606369D4
:106D9000D36094F8633003B3012B4FF480710CBFC0
:106DA0004FF4007300230B4394F86210104602293D
:106DB0000CBF402100210B4343F03003936094F853
:106DC0005A10002914BF4FF0004100210B4393607B
:106DD000D4F85E10FDF7C4FDB7E71946E3E7002AD3
:106DE00000F09D801368E36053682361D36863619A
:106DF000936894F85A20B2EBD37FA6D0002B18DB0F
:106E000094F859309A0712D443F00303204684F8CB
:106E10005930FFF784FD054600232046A4F85A3078
:106E2000FFF7BCFD012384F85D30284638BD0025FE
:106E3000F2E70123A4F85A3094F85C307BB194F85F
:106E40005930204623F0020343F0010384F85930FF
:106E5000FFF765FD0123054684F85B30E2E7002576
:106E6000E0E7EFF3118000238021EFF3108372B687
:106E700081F3118883F31088218EE38D09B21BB250
:106E8000994208DCE38D218E1BB209B25B1AC1B2B4
:106E900081F311886BE7218EE58D09B2B4F93230A8
:106EA0002DB2491BF2E7EFF3118000238021EFF3AD
:106EB000108372B681F3118883F31088A18C638CE0
:106EC00009B21BB2994203DC638CA18C1BB2DCE7D4
:106ED000A18C658C09B2B4F926302DB2E1E7EFF34D
:106EE000118000238021EFF3108372B681F31188A3
:106EF00083F31088618CA38C09B21BB2994206DA25
:106F0000A38C618C1BB209B25B1A013BBFE7618C99
:106F1000A58C09B2B4F926302DB2491BF4E76FF005
:106F2000150582E770B50D46044658B151B10868A1
:106F300008B1FDF7B9F8236829462046DB68BDE8AB
:106F40007040184770BD10B590F85430044693B1A6
:106F5000002180F85410FFF76DFBE06E03685B685A
:106F60009847206F03685B689847606F0368BDE8C7
:106F700010405B68184710BD70B50C468568EFF38C
:106F8000118600238022EFF3108372B682F31188FA
:106F900083F3108800212846FFF74CFB2846FFF7B3
:106FA000D2FF0023F6B26B84AB8486F3118823688A
:106FB0005B6923B120460121BDE87040184770BDD0
:106FC0002DE9F04184680D46002C49D02046FFF79A
:106FD000BAFF3220FDF744F8E16E29B12B6828464C
:106FE0005B6898470023E366A16F21B16868FFF7EB
:106FF00099FF0023A367264604F130074FF00008ED
:10700000D6F8E81021B1606FFFF78CFFC6F8E88072
:107010000C36BE42F4D1616F29B12B6828465B68FB
:10702000984700236367EFF3118600238022EFF374
:10703000108372B682F3118883F3108804F18C08F0
:10704000D4F88C7077B9F6B286F31188216F21B12C
:107050002B6828465B689847276700236384A384CE
:10706000BDE8F0814046FDF7DDF941680029E7D031
:10707000206FFFF757FF94F85530013B84F85530E7
:10708000DEE7FFEC2DE9F84F84680D468046216568
:107090004B6840219C606868FFF71EFCA0670028D1
:1070A00079D03E4B0122C36028462B6894F8B0107B
:1070B0001E68032341F08001B047E06630B96FF0ED
:1070C000120429464046FFF77BFF61E084600122FD
:1070D0002B68284694F8B4101E68022341F0800102
:1070E000B04720670028EAD0846000222B68284639
:1070F00094F8B8101E680223B04760670028DED0FD
:1071000004F1E40604F58A7A4FF0000B8460B1467E
:107110004021606FFFF7E0FB706000283BD0A6F8CD
:1071200008B006610C3656F8082C1D4B5645D36046
:10713000EED104F1C4064FF0800A6021206FFFF702
:10714000CBFB706038B30661164A7368DA60EFF300
:10715000118BEFF3108772B68AF3118887F31088CA
:1071600004F18C013046FDF73DF994F855205FFAA3
:107170008BF3013284F8552083F3118808364E458D
:10718000DBD12B685C691CB101212846A047002493
:107190002046BDE8F88F6FF00B0492E7AF68000857
:1071A000A16A00089D6C000837B5044615460846DC
:1071B0001A466946002300F039FA23682A466946D0
:1071C0001B682046984703B030BDFFEC2DE9F34122
:1071D00090F8543004460E468B4204D100252846D0
:1071E00002B0BDE8F081FFF7AEFE002EF6D0012E12
:1071F00041D1002204F19C03E06E11460193FFF798
:10720000D3FF051E33DBE26E0221019B9460002256
:10721000206FFFF7C9FF051E29DB226F3146019B56
:1072200094603246606FFFF7BFFF051E1FDB636F80
:10723000264604F13007DFF844809C60D6F8E81059
:10724000C1F80C80606F03681B699847054670B9E8
:1072500094F856300C360133BE4284F85630EDD1E6
:107260000121204684F85410FFF7E4F9B7E72046DF
:10727000FFF769FEB3E76FF01505B0E7A16A0008F4
:107280002DE9F8430F4692F804C0517996794CEAFB
:10729000012CD179D0F8088092F8039046EA0126B3
:1072A0009078117840EA092ED8F8785011F06004EF
:1072B0000FFA8EFE7FD153781FFA8EF4063B052B12
:1072C00000F2CD80DFE803F003CB433A654CB9F11F
:1072D000020F26D0B9F1030F2CD0B9F1010F40F005
:1072E000BE802C6800F09EF900F11002234650F891
:1072F000041B904243F8041BF9D1028812201A8023
:10730000B0424FF001032946A8BF30462B71E880F8
:10731000786803681B699847002809DA00236B81A5
:1073200006E008F19C01286800F0B6F90028E7DAC9
:10733000BDE8F883296800F039F9F7E7002940F043
:107340008E805FFA8EF14046FFF740FFEEE780291E
:1073500040F085802B6898F854201A700120CFE700
:1073600001297CD198F85430012B78D1D8F8A0307D
:107370009C4502D001339C4571D1002C6FD1404611
:10738000FFF7E1FD98F854104046FFF71FFF00207B
:10739000B6E7812963D198F85430002B5FD1D8F833
:1073A000A0309C4502D001339C4555D1002C53D1CF
:1073B0002B681C70D2E7202C51D15278203A032A36
:1073C0004DD8DFE802F014022D3DA12947D1D8F8AD
:1073D000A0309C4543D158F85E2F07202B681A60D7
:1073E000B8F804209A8098F806209A7188E7212935
:1073F00035D1072E33D1D8F8A02094452FD143B1F1
:107400001A68C8F85E209A88A8F862209B7988F8E4
:107410006430D8F86830002BB9D000209847B6E720
:1074200021291CD1D8F8A0309C4518D10EF0030EAC
:10743000D8F8683088F858E0002BA8D00120EDE794
:1074400021290CD1D8F8A0309C4508D1D8F8683053
:10745000002B9CD00220E1E76FF0200068E76FF07E
:107460005E0065E77047FFEC2DE9F04F8FB02422F6
:1074700007460E4605A80021FDF7ECF94FF002097A
:1074800004234FF0030B4FF0010A43F25820CDF8CC
:1074900010900693CDE908BACDE90A9BFCF70CFEE3
:1074A000044638B96FF00B0706B1346038460FB0A8
:1074B000BDE8F08F43F24C28002100254246FDF73D
:1074C000C9F90DF1100E04F19C0C84F85770BEE858
:1074D0000F00C4E92355C4E92555ACE80F00BEE808
:1074E0000F00ACE80F009EE803004FF442431E4A31
:1074F0008CE80300A4F85E300823C4F860A01021D3
:1075000084F864304FF4167384F803A004EB080A7F
:10751000638604F58A7384F859B06846636342F65B
:10752000E063E38404F55B73A362104BC4E90E349B
:107530000F4B8AF8049044F808303B46CAF80840DC
:1075400001F05DFC21466846FEF726FF071E04DABF
:1075500020462C46FCF7A8FDA6E750465446FCF70B
:1075600081FB0746A0E700BF78A10008A0A10008A2
:1075700088A1000830B585B085680B4A102195F8C0
:1075800057300446684601F03AFC684600F0A9FE10
:107590002046FCF781FB05F17C00FAF7E3FC284666
:1075A000FCF782FD05B030BD78A1000870B50C462F
:1075B00004282BD8DFE800F01521031D1F00154D0E
:1075C0002846FDF7B2F90023A21C1946834202F1B6
:1075D000020214DB4000032302306370C0B220704B
:1075E00006E0032304204B70092308708B70C870D9
:1075F00070BD094DE4E7094DE2E7094DE0E7EE5CB7
:10760000013302F8011C02F8026CDFE76FF015008D
:10761000EEE700BFE1A1000857A20008D4A10008CE
:10762000D9A1000800487047FBA10008012810B547
:1076300012D002281FD068BB072305240B704C70A2
:107640005269487162F07F028A700322CA70402238
:107650000A710A228A710CE0072305240B704C7012
:10766000D26988718A700222CA7040220A7100228F
:107670004A71184610BD072305240B704C7092699F
:10768000C87062F07F028A7040220A7100224A713B
:107690000122DFE70023ECE72DE9F0410D46044627
:1076A000002800F087800021042624274FF00308DB
:1076B0000846FFF7F1FF8023012102224FF0090E57
:1076C000A070E3710012FA23A671E0704FF0100C65
:1076D000A672052084F800E0627022716171237245
:1076E00084F809E06B6884F815C04FF0060CE3726B
:1076F0000023A074E67584F81AC04FF0070CE076FA
:1077000084F81E8023736173A273E273217463741F
:10771000E7742375A17527766276277761776F689E
:1077200084F820C00F4484F82100E7776F6984F85B
:1077300023804FF00A0867F07F0784F8253084F82B
:10774000268084F82270402784F827E084F824708B
:1077500084F828606E6884F82A300E4484F82B2060
:1077600084F82C8084F8296084F82D3084F82E3039
:1077700084F82F3084F830C084F83100EE6984F842
:10778000332084F8326084F8347084F8353084F81B
:10779000361084F837C084F83800A86960F07F009C
:1077A00084F8390084F83A2084F83B7084F83C303F
:1077B00084F83D103E20BDE8F08110B5144608461F
:1077C000114601F0ADF9204610BD0846FBF7CEB9D1
:1077D00000F042B9F8B5837804460E468B4223D2B6
:1077E000CB00FF2B22D88900406801F0A7F907469B
:1077F00068B1A5788020FCF767FC47F8250070B9D0
:10780000013DA3789D4205DA3846FCF74DFC6FF048
:1078100016000AE057F82500FCF746FCF0E70135B2
:10782000B542E7D36760A6700020F8BD6FF017007F
:10783000FBE701220021FCF73EBEF8B5044685783F
:10784000013D07D26068FCF72FFC2046BDE8F840F8
:10785000FAF789B9AF0070266368D8593044103EF2
:1078600000F020FA16F1100FF6D16368D859FCF732
:107870001BFCE5E72DE9F84FDDF828A08846174600
:107880001D46064600F0D0FD814600F0A5FE041E10
:107890003EDBBAF1000F514699F80230B8BF0AF149
:1078A0000701C9108B428B4609DC01314846FFF7BE
:1078B00091FF041E03DA484600F0A4FE28E0DAF146
:1078C00000030AF00704D9F804C003F0070358BF07
:1078D0005C425CF82B204FEA8B0102EB04129368A8
:1078E0002001D3B9C2F8008004EBCB04D9F80420FE
:1078F000535803445F60D9F804305B5803449E60DA
:10790000D9F804305B5803444846DD6000F07AFE45
:107910002046BDE8F88FD346DBE701341032082C4F
:10792000DDD10BF1010A99F8023000245345F2DC55
:107930000BF102014846FFF74DFF041EBBDBD9F8EF
:1079400004304FEACA0453F82A30C3F80080D9F84B
:10795000043053F82A305F60D9F8043053F82A30E5
:107960009E60D9F8043053F82A30DD60A3E7F8B5FB
:10797000002305460F460B6000F056FD0646F0B1A9
:10798000002D1FDB8378B5EBC30F1BDA00F024FE5C
:10799000041E0FDB7368EA1005F0070553F8220098
:1079A00000EB05153D60AB6833B12B4630463B60BC
:1079B00000F028FE2046F8BD6FF00804F6E76FF0EF
:1079C0000A04F7E76FF00804F4E7F0B585B0044661
:1079D00000F02AFD054600F0FFFD002814DB002C16
:1079E0000DDBAB78B4EBC30F09DAE2106B6804F07F
:1079F000070453F8220000EB0414A36833B92846A7
:107A000000F000FE6FF0080005B0F0BD23466E46A2
:107A100004F110071868083353F8041C3246BB42BF
:107A200003C21646F6D1102200212046FCF712FFB1
:107A3000284600F0E7FD684600F034F9E4E710B5A9
:107A4000FFF7C3FF041E05DA6442FCF7C1FC0460C3
:107A50004FF0FF34204610BD00F05CB870B500F068
:107A6000DBFE0F4B04465A681D46904212D01E465C
:107A7000304600F0B9FD002807DAFCF7A9FC0068E1
:107A80000428F5D08C28F3D0404238B901236C602B
:107A90002B8103E01A89002001321A8170BD00BFDA
:107AA0008400002408B500F0B7FE0A480389012BC2
:107AB0000CD1002303814FF0FF33436000F0E0FD61
:107AC000002805DABDE80840FCF782BC013B0381D1
:107AD00008BD00BF8400002410B5034604461846C4
:107AE00013F8012B2AB9001B1C30FCF7EDFA18B96A
:107AF00010BD2F2AF3D1F6E700F11803013C14F86A
:107B0000012F12B900221A70F2E72F2AFAD003F8D7
:107B1000012BF4E708B50348FFF7DEFF024B1860BE
:107B200008BD00BF149E0008E013002400232DE9C7
:107B3000F04116461360027888B0002A45D08DF8CF
:107B40001C30CDE9010301A8CDE90333CDE90533AC
:107B500000F04CF8002835DA019FDDE9035438467F
:107B600000F036F8037880463846D3B1FFF7B4FF0B
:107B700048B96FF00B04069808B1FCF795FA204657
:107B800008B0BDE8F0813DB16B68C0E900436860B2
:107B9000474604460025E2E7A368C0E90043A06029
:107BA000F6E7FFF799FF0028E3D035B16B68C0E92D
:107BB0000043686000243060DDE7A368C0E900434B
:107BC000A060F7E76FF01004D5E76FF01504D6E773
:107BD000017803460246013031B12F29F8D113460E
:107BE000013219782F29FAD018467047F8B5036882
:107BF00005461A782F2A08D0274A1430274901F061
:107C0000F1F86B69002B41D02B60254B28681C686C
:107C100003782F2B3DD1002637464CB922466FF012
:107C200001032A61C5E90004C5E902761846F8BDDA
:107C300004F11701431E11F801CF13F8012FBCF115
:107C4000000F0FD10AB12F2A17D1FFF7C1FF037818
:107C5000BBB1E38903F00F03032B14D0A3682646BE
:107C600000240BE022B12F2A02D0944505D3E2D99B
:107C700000246FF001032246D3E7636827461C46C1
:107C8000CBE70246CDE702460023CAE76FF00B03BD
:107C9000CCE76FF01503C9E7149E000824A2000882
:107CA000E013002470B5866805467EB134691CB1C6
:107CB00064680CB1A0470446304600F043FB002343
:107CC000C5E90033C5E90233204670BD3446FBE701
:107CD00070B5866804460B4615463EB136692EB12E
:107CE00036691EB1B04700280DDA70BD012D05D0F0
:107CF000022D0AD025B16FF01500F6E76268134433
:107D0000002BF8DB63606068EFE76FF05700ECE78B
:107D10001FB50C4603A90192FFF729FE002804DBDA
:107D2000019A21460398FFF7D3FF04B010BD10B5A8
:107D3000FFF7EEFF041E05DA6442FCF749FB04601E
:107D40004FF0FF34204610BDC38913F00F030FD04E
:107D500003697BB1CA0701D59A6872B111F00200BC
:107D60000DD0DB68002B14BF00206FF00C007047B3
:107D7000184670476FF0050070476FF00C007047B1
:107D80002DE9F047054688B09246984600295BD019
:107D900012F0060F4FF0000601A8019114BF109BCE
:107DA0004FF4DB79069618BFD3F800908DF81C606D
:107DB000CDE90266CDE9046600F0B1FA041E19DBD4
:107DC000029F51463846FFF7BFFF041E0DDB1AF431
:107DD000006FC5E900A6C5E9027610D005992846CE
:107DE00000F0BAF90028044611DA00233846AB60E7
:107DF00000F0A8FA069868B1FCF756F90AE0FB898A
:107E000003F00F03032B10D13B691C6834B90698AB
:107E1000A0B90024204608B0BDE8F08729EA08038D
:107E2000524605992846A047DCE7012B09D13B695A
:107E30001B68002BEBD028469847D3E7FCF734F9B2
:107E4000E7E76FF00504D0E76FF01504E2E770B5DF
:107E5000044686B00D46164600F076FF21460346DE
:107E60002A4602A80096FFF78BFF041E0CDB0023B6
:107E700004980093059BDDE90212FFF7FBFC041E4A
:107E800002DA02A8FFF70EFF204606B070BD0EB45E
:107E900017B505AA52F8041B0192FFF7D8FF041E7C
:107EA00005DA6442FCF794FA04604FF0FF34204690
:107EB00003B0BDE8104003B0704710B40368846895
:107EC000DB0707D55CB123694BB19B683BB15DF81B
:107ED000044B18476FF00C005DF8044B70476FF0CF
:107EE0000800F9E71FB50C4603A90192FFF73FFD13
:107EF000002804DB019A21460398FFF7DEFF04B057
:107F000010BD10B5FFF7EEFF041E05DA6442FCF762
:107F10005FFA04604FF0FF34204610BD10B40468CF
:107F2000A40708D583685BB11B694BB1DB683BB123
:107F30005DF8044B18476FF00C005DF8044B704778
:107F40006FF00800F9E71FB50C46019259B103A97B
:107F5000FFF70DFD002804DB019A21460398FFF787
:107F6000DDFF04B010BD6FF01500FAE710B5FFF7A4
:107F7000EAFF041E05DA6442FCF72AFA04604FF0B7
:107F8000FF34204610BDB1F5417F08B5C36805D167
:107F900059681046FCF7A5FC002008BD6FF01800DA
:107FA000FBE770B5C56806460C462868002956D020
:107FB000212A54D9C38903F00F03032B0BD1036982
:107FC0000A4629465B6B9847002844DB73682220E9
:107FD0000133736042E0A96800293ED021221831A4
:107FE000601CFCF786FC00232370AB681A6932B171
:107FF000DB8903F00F03022B17D106232370AB6834
:108000009A680AB91B690BB904232370FFF726FD90
:10801000AC686368AB6013B19A8901329A81FFF74B
:1080200041FD204600F08EF9D0E7072B01D109234E
:10803000E4E7032B01D10423E0E7012B01D1022364
:10804000DCE7042B01D10323D8E7052BD6D0062B80
:10805000D5D10723D2E7831C00D1002070BD6FF07B
:108060001500FBE770B5C468D4E90056EB8903F04E
:108070000F03032B0ED12B691B6BA3B1214628469E
:1080800098470446284600F05DF93046FCF70CF8A6
:10809000204670BDA06808B100F054F920460024C5
:1080A000FCF702F8EEE71C46ECE72DE9F043064644
:1080B0008BB089461746002A48D1D0F80C80446816
:1080C000D8F80050EB8903F00F03032B20D1A14215
:1080D0000CDA2B699B6B2BB96FF0850420460BB033
:1080E000BDE8F0833C464146284698472746B945B7
:1080F00004DC3C46002CF1DB7460EFE72B6901AA3D
:10810000414628465B6B9847041EE7DB0137EEE7E4
:10811000A142BABFAD681446D8F80850FFF79EFCDC
:108120000DB1A1450FD1D8F80870C8F8085015B1A5
:10813000AB890133AB81FFF7B5FC002FDAD03846AD
:1081400000F000F9D6E701346D68E9E7012A0CBFB9
:1081500044686FF01504C1E7F7B5856806460F4619
:10816000EB8903F00F03032B19D12B6923B3DC6ACE
:1081700014B35B6B03B301AA2846A047041E0BDBB4
:10818000019B1D60019D384600F0BEFE68600D48F1
:10819000C6E9020500F0B3F8204603B0F0BD0C209C
:1081A000FBF792FF034650B1019000240560A868D8
:1081B000986000F0A4F8E5E76FF05704ECE76FF083
:1081C0000B04E9E790000024C3685968FFF7C4BFB7
:1081D0002DE9F347061E884614461F4659DB12B99F
:1081E00000F0A2F90446022E16DD01A93046FFF781
:1081F000BEFB051E04DB019B986830B96FF00105DA
:10820000002F3AD000233B6037E04146FFF79CFD4A
:1082100010B16FF00C05F3E7022ED4F8089033DDAF
:108220004C20FBF751FF0446B0B309F12C0A50462D
:1082300000F0A2F9051E03DA2046FBF735FFDFE761
:10824000D9F81831EBB11C605046C9F8184100F05C
:10825000D9F92046FCF783FA04F1240304F144021F
:10826000666063612362A4F84480C4E906230C239A
:1082700084F846309FB100253C60284602B0BDE836
:10828000F087C9F81441DFE74C2404FB069430342E
:10829000E2E76FF00805B3E76FF00B05B0E73D4686
:1082A000EBE7F0B585B007460E461D460192FFF795
:1082B000D5FB041E12DB03AA01993846FFF736FCF2
:1082C000041E09DB039B0024DA8922F00F0242F02E
:1082D0000102C3E90465DA81FFF7E4FB204605B03B
:1082E000F0BD38B50546FFF7B9FB041E05DB28468F
:1082F00000F06BF80446FFF7D5FB204638BD38B5D3
:10830000044650B1FFF7AAFB051E04DBA389013325
:10831000A381FFF7C7FB284638BD0546FBE738B504
:108320000546FFF79BFB041E0ADB2846FFF75EFCB1
:10833000041EA1BF6A68938901339381FFF7B2FBE2
:10834000204638BD10B50446C8B1FFF787FB0028AA
:10835000FBDBB4F90C304BB9E389DB060BD5FFF737
:10836000A1FB2046BDE8104000F044B8013B1BB221
:10837000002BA381F0DDBDE81040FFF793BB10BDDB
:1083800010B5044688B0D0B100240123019001A8A3
:1083900006948DF81C30CDE90244CDE90444FFF782
:1083A00025FCA04207DBDDE90242636852B153605D
:1083B0000023C4E90033069808B1FBF775FE204698
:1083C00008B010BD049A9360F2E710B5FFF7D8FF2C
:1083D00068B1B0F90C4034B1C28942F01002C281D8
:1083E0006FF00F0010BD00F005F82046FAE76FF0BF
:1083F0000100F7E710B5044650B14068FFF7FAFFF7
:10840000A068FFF7F7FF2046BDE81040FBF74CBE21
:1084100010BD00F06BBBFFEC024A13680133136020
:10842000704700BFE4130024024B1B68986800B13A
:1084300024307047BC0300240F4B10B51B68044662
:10844000B3F92020002A0ADD1A7C037C9A4206D266
:108450000A49F9F7DDFD01230020237710BD064905
:108460002046F9F7D5FD022320B1032222772268A6
:108470001377F3E72377F1E7BC030024B00300246C
:1084800038B5436804465BB90368032201251A77AF
:1084900020460449FBF7F6FF00232846237738BD22
:1084A0000025F5E7BC030024F0B513490020134C68
:1084B0000226032722680B681BB90B604B60F0BDD6
:1084C0001268B2B193F810C0157CAC45F8D9556864
:1084D000D3F800C0C3E900253DB9012053601677E9
:1084E00023601F771A466346E6E72B6053601E77CA
:1084F000F8E75368FFDE00BFB0030024BC0300248C
:10850000024B1B6898682C30704700BFBC030024E6
:10851000044B1B6823B11868B0FA80F0400970471B
:1085200001207047BC030024014B1868704700BF4E
:10853000BC03002438B50F4B0C461D6870B1F9F729
:10854000B9FAA0B1EB8B03F00303022B07D0AA68A2
:1085500083689A4203D06FF00C0007E02846436B13
:108560002360836B6360C36B0020A36038BD6FF032
:108570000100FBE7BC03002438B5164B1C68EFF381
:10858000118500238022EFF3108372B682F31188E5
:1085900083F31088D8B103881BB2002B038803F142
:1085A000FF331BB2038005DD00202064EDB285F3AC
:1085B000118838BD00232064052120466384F9F723
:1085C000C5FEB4F922000028F0D04042EEE76FF07B
:1085D0001500EBE7BC03002410B504462046FFF766
:1085E000CBFF031DFAD010BD10B5FFF7C5FF041E69
:1085F00006DA6442FBF7ECFE04604FF0FF3010BD7A
:108600000020FCE738B5002834D0EFF311850023B3
:108610008022EFF3108372B682F3118883F31088FF
:10862000038847F6FF721BB2934205D1EDB285F382
:1086300011886FF08A0038BD038801331BB20380B4
:1086400003881BB2002B0EDC0C4B1C685CB1236C46
:1086500083420DD104F12400F9F784FC0023204665
:108660002364F9F749FFEDB285F311880020E2E7B2
:108670002468EBE76FF01500DDE700BFD0030024AE
:1086800010B5FFF7BFFF041E05DA6442FBF7A0FE3A
:1086900004604FF0FF34204610BD70B505460C460F
:1086A000F8F7E0FBEFF3118600238022EFF310834D
:1086B00072B682F3118883F310882B881A0409D4C8
:1086C0002B881B040ED5F6B286F31188F8F7DAFB77
:1086D000002070BD002CF3DD013C2846FFF792FF1F
:1086E00024B2EAE72C80EEE737B5041E0D4616DB10
:1086F0001F2917D8F8F7B6FB002304222046694645
:108700008DF800508DF801308DF802200193F9F7B3
:108710005BF80446F8F7B6FB204603B030BD6FF0B7
:108720005704F9E76FF01504F6E7FFEC07B568B1F9
:10873000084A0021B0FBF2F302FB130000934FF450
:108740007A7358430190684600F0F0F803B05DF882
:1087500004FB00BF40420F0038B50F4C2568284687
:10876000FFF78EFE0D4B1B680BB1FFF79DFE2468D3
:1087700028460421238C0133238402232377F9F72D
:1087800025FC0121E86800F019F803232377238CE6
:10879000013B238438BD00BFBC030024B003002488
:1087A000054B186830B1037F032B01D1C0687047B7
:1087B0006FF00200704700BFBC03002470B50E4686
:1087C000EFF3118500238022EFF3108372B682F35A
:1087D000118883F31088F9F76DF90446EDB2A0B162
:1087E000027F0C4B53F83210FBF74CFE85F31188D7
:1087F000002120463246F9F701F9A17F204601F019
:108800000301BDE87040F8F7B5BD85F311886FF03E
:10881000020070BDB49C0008054B186830B1037F9E
:10882000032B01D1C06870476FF00200704700BF92
:10883000BC0300242DE9F0410C4616469846054637
:10884000002839D0002A37D0002935DBEFF3118713
:1088500000238022EFF3108372B682F3118883F332
:10886000108843680BB1F9F77DFB1F4901346E6036
:108870000E68C5F80C801EB92846FBF7B3FD2CE046
:1088800030463246002391685B1801D5116831B932
:10889000A34214DC116829B9E41A1349ECE7104625
:1088A0000A46F0E78868034410460A46F0E70E4A95
:1088B000294600F054FA10E06FF0150012E09168BC
:1088C0009642A3EB0103A4EB0304A1EB0401916026
:1088D000EDD10549284600F03CFAAC60FFB287F3C1
:1088E00011880020BDE8F0813809002470B50E4CD5
:1088F00023684BB19A6825460026013A9A6023689E
:1089000013B19B68002B00DD70BD2846FBF78AFD84
:1089100023681BB19A6881680A449A60436846607C
:10892000C0689847EBE700BF380900242DE9F743FA
:108930000F46054600283BD042681F4B9A4237D865
:10894000EFF3118600238022EFF3108372B682F3D7
:10895000118883F31088DFF864906846F6B2D9F87E
:108960000080FBF7F4FD2A460021684600F038F845
:1089700010F10B0F044606D186F31188002420461F
:1089800003B0BDE8F08387B101A9284600F004FADE
:10899000D9F8003001983946A3EB080290428ABF0B
:1089A000C01A0020404400F0E9F986F31188E6E798
:1089B0006FF01504E3E700BFFFC99A3BE4130024FE
:1089C000027F062A0AD140F2FF22A0F85C2074221E
:1089D00080F85E2000220266F9F78EBD7047FFEC3A
:1089E0003A4B2DE9F74306460D4691461C68EFF3D6
:1089F000118800238022EFF3108372B682F311886E
:108A000083F3108807682046F9F724FA38405FFAA4
:108A100088F70190B0B101A8F8F798FD014620460B
:108A2000F8F742FD2DB1024652F8043F2B6053681F
:108A30006B600679F8F75CFD87F31188304603B068
:108A4000BDE8F0833368A364B9F1000F33D0D9F8DF
:108A5000043000211E4804F12408D9F800E0C018B1
:108A6000DFF878C01B4A41EBE3710023ECFB0E01F9
:108A700000F0F4FA23460146174A4046FFF7DAFEB3
:108A800020460621F9F762FC4046F9F76BFA94F8A4
:108A90005C1000231F29A36412D83046FBF75BFD4E
:108AA00088B194F85C60002DC6D054F85C3F2B6010
:108AB00063686B60C0E706212046F9F747FCE6E7EC
:108AC0006FF00A06EFE76FF00306ECE7BC03002443
:108AD0003F420F0040420F00C189000800CA9A3B84
:108AE00008B500F05DFA002008BDFFEC08B5084AA3
:108AF0000F20084B08491A6000225A60F8F75AF90B
:108B0000064B07220F201A60BDE80840F7F714BF94
:108B1000FF52070014E000E0E18A000810E000E0E6
:108B200070B504460E46451E15F8010F10B1731BB3
:108B3000DC4200D170BDFAF719F8F5E7024B0A469E
:108B40000146186800F002B8B00E00242DE9F84F75
:108B5000814614460F4621B91146BDE8F84FFBF790
:108B6000CBBB12B9FBF76CFB18E002F1170525F03F
:108B70000F05AA4200F2B480A1F10806FBF70CFB36
:108B800057F808AC55450CD804D22A463146484619
:108B900000F0A8F83C464846FBF722FB2046BDE81B
:108BA000F88F57F8041C06EB0A0B21F00101DBF8E3
:108BB0000430711ADA074B684CBF4FF0000856F8C2
:108BC0000A80DB0708EB0A0354BF0868002003444F
:108BD000AB4272D34045A5EB0A054DD2A84251D213
:108BE0002D1A0246002A60D0D1E902439C600CB1E4
:108BF000CB68E3609042A6EB020646D90B689B1A4D
:108C000052440B603260086840F0010070604846D2
:108C1000DBF8043003F001031A43CBF80420FBF720
:108C2000E7FA06F10804DDB10BEB0800DBE90223EB
:108C30009A6012B1DBF80C30D3603368A8452B443E
:108C4000336034D9A8EB0505F118F55033684B6053
:108C5000436803F001031D4345604846FBF7C8FA2B
:108C60004846FBF7BDFABC4298D0AAF10802394643
:108C70002046F7F7BDFE91E7A84516D2A5EB0802FE
:108C80004546AFE72A460025ACE733680AEB030206
:108C9000736843F0010332607360DBF8043003F063
:108CA00001031343CBF80430BBE73C46BBE7426803
:108CB00002F0010213434360D2E74846FBF790FA03
:108CC00021464846FBF718FB044600283FF466AFF0
:108CD0003946AAF10802F7F78BFE3946484641E7C4
:108CE00000245BE7F0B40C680B4606460D19696872
:108CF000C90719D41859D5E902172844B96009B130
:108D0000ED68CD601D6899181C59AD1A25449D5019
:108D10004A601A6044689B5804F001041C43446094
:108D20003046F0BCFBF764BA02F110018C4209D363
:108D30009918A41A9C504A601A609B5843F001038A
:108D40006B60EEE7F0BC704708B500F023F9406BAC
:108D500008BD0B68036003B94860086070470346AC
:108D600008461146126812B14A689A4201D1FBF7CF
:108D700039BB1A68026018607047FFEC4FF47A72D2
:108D800090FBF2F302FB13000B60024B4343002005
:108D90004B60704740420F0070B544680E46026851
:108DA0000021084BE5170848E3FB0245074A201855
:108DB0004FF0000345EB010100F000F930600020A6
:108DC00070BD00BF00CA9A3B3F420F0040420F00F7
:108DD000084631B10139022934BF6FF085006FF0C8
:108DE000150070470EB403B503AA52F8041B019294
:108DF00000F01DF802B05DF804EB03B070470CB44E
:108E00000A4600B589B071B1014602A800F058F8D1
:108E10000BAA0A9902A80192FBF7F2FD09B05DF8CE
:108E200004EB02B0704702A800F062F8F0E770B5FA
:108E30008EB014460D46064604A8039200F058F87A
:108E40002246294604A8FBF7DBFD079A01321046AB
:108E50000192FBF731F9044660B10146019A08A876
:108E600000F02EF8039A294608A8FBF7C9FD3460E4
:108E70000EB070BD4FF0FF30FAE738B50546C06858
:108E80006B691B1A934228BF1346002B1C460ADD50
:108E90002B6922461844F7F7ABFDEB682A690021DD
:108EA0002344EB60D154204638BD07B501228DF82C
:108EB00007100DF10701FFF7E0FF03B05DF804FBB9
:108EC000064B013A0360064B42614360054B8360E9
:108ED0000023C0E903310B70704700BFAB8E000860
:108EE0007B8E000883540008C3680133C360704759
:108EF000034B0360034B83600023C360704700BFD4
:108F0000E98E00088354000813B50190FBF70DFDAE
:108F10000130FBF7D1F8044610B10199FBF7E1FCF1
:108F2000204602B010BDFFEC014A00F003B800BFBC
:108F3000E81300242DE9F04188461646044610B98E
:108F4000CAB11468BCB125462C4615F8011BA9B15D
:108F5000404600F015F80028F6D129782F46013553
:108F600039B1404600F00CF80028F6D000233B70E1
:108F70002F4606B137602046BDE8F0810C46FAE77F
:108F800003461A78184601338A4202D0002AF8D1E3
:108F90001046704708B5FBF705FD006808BDFFECFB
:108FA00008B5054B0BB1FFF737FAFFF79FFCBDE89B
:108FB0000840F7F73BBE00BF198400087BB972B9BF
:108FC0000029BEBF00204FF0004106E008BF002886
:108FD0001CBF6FF000414FF0FF3000F0DBB9ADF186
:108FE000080C6DE904CE002909DB002B1ADB00F028
:108FF0006FF8DDF804E0DDE9022304B07047404279
:1090000061EB4101002B1BDB00F062F8DDF804E0AE
:10901000DDE9022304B0404261EB4101524263EBBF
:1090200043037047524263EB430300F051F8DDF80D
:1090300004E0DDE9022304B0404261EB41017047E6
:10904000524263EB430300F043F8DDF804E0DDE94E
:10905000022304B0524263EB4303704753B94AB949
:10906000002908BF00281CBF4FF0FF314FF0FF3030
:1090700000F090B9ADF1080C6DE904CE00F028F8CD
:10908000DDF804E0DDE9022304B07047FFECC29292
:109090009FED0B6B41EC170B9FED0B5B27EE066B07
:1090A000BCEEC66BB8EE464BA4EE457BFCEEC77B30
:1090B00016EE101A17EE900A704700BFAFF300804B
:1090C000000000000000F03D000000000000F04142
:1090D0002DE9F047089D04468C46002B40F0838024
:1090E0008A42174647D9B2FA82F242B1C2F1200051
:1090F00024FA00F09140974040EA010C94404FEA76
:109100001748230CBCFBF8F61FFA87FE08FB16C1B4
:1091100043EA014306FB0EF1994209D9FB1806F117
:10912000FF3080F01981994240F21681023E3B44A3
:109130005B1AA4B2B3FBF8F008FB103344EA034413
:1091400000FB0EFEA64509D93C1900F1FF3380F063
:109150000581A64540F2028102383C4440EA0640BF
:10916000A4EB0E0400261DB1D4400023C5E9004342
:109170003146BDE8F08702B9FFDEB2FA82F2002A7A
:1091800050D1CB1B4FEA174E1FFA87F80126B3FBCD
:10919000FEFC210C0EFB1C3341EA034108FB0CF3DF
:1091A0008B4207D979180CF1FF3002D28B4200F2C2
:1091B000E9808446C91AA3B2B1FBFEF00EFB101180
:1091C00043EA014408FB00F8A04507D93C1900F127
:1091D000FF3302D2A04500F2D9801846A4EB080460
:1091E00040EA0C40BFE78B4209D9002D00F0B18066
:1091F0000026C5E9000130463146BDE8F087B3FAE4
:1092000083F6002E4AD18B4202D3824200F2B8800C
:10921000841A61EB030101208C46002DA8D0C5E91A
:10922000004CA5E7C2F1200320FA03F6974001FAAB
:1092300002F04FEA174ED9403043030CB1FBFEF663
:109240001FFA87F80EFB161143EA014306FB08F1EB
:10925000994204FA02F409D9FB1806F1FF3C80F0A8
:109260008D80994240F28A80023E3B445B1A81B273
:10927000B3FBFEF00EFB103341EA034100FB08F3A1
:109280008B4207D9791800F1FF3C73D28B4271D918
:1092900002383944CB1A40EA064678E7C6F1200C7A
:1092A00003FA06F422FA0CF31C4320FA0CF701FA35
:1092B00006F34FEA144E21FA0CF11F433B0CB1FBAD
:1092C000FEF91FFA84F80EFB191143EA014109FB6C
:1092D00008FA8A4502FA06F200FA06F308D961187C
:1092E00009F1FF3048D28A4546D9A9F10209214443
:1092F000A1EB0A01BFB2B1FBFEF00EFB101147EA71
:10930000014700FB08F8B84507D9E71900F1FF311C
:109310002ED2B8452CD90238274440EA0940A7EBA1
:109320000807A0FB02894F45C64649461AD317D005
:109330005DB1B3EB0E0267EB010707FA0CFCF240DC
:109340004CEA0202F740C5E9002700263146BDE895
:10935000F0872E4628460BE70646E9E61846FDE666
:109360004345E5D2B8EB020E69EB04010138DFE7B3
:109370000846D2E760468DE78146B9E7664675E75D
:1093800030464AE7ACF1020C394413E702383C445A
:1093900024E700BF704700BF0720704710B50820C2
:1093A000064CF8F7ADFE4FF0006322202360F8F77B
:1093B000A7FE0023024A2360136010BD80440258B8
:1093C000D844025808B5042000F08AF9064B4FF43F
:1093D0007A70DB68584300F077F900F0A7F9BDE830
:1093E000084000F08DB900BFAC00002408B500F0C3
:1093F000A5F900F08DF9002000F072F90020BDE819
:10940000084000F061B9FFEC0C4B1A6842F0010211
:109410001A601A685207FCD5094A002111601A68BF
:10942000084922F0A85222F410221A60064A11605C
:109430001A6822F480221A60704700BF0044025864
:10944000104402580000FF012C44025808B54FF0A8
:10945000006000F008FA4FF00160BDE8084000F03D
:1094600002BA08B500F08AFB4FF0006000F0E8F99E
:109470004FF00160BDE8084000F0E2B900F09CBA8E
:10948000014B1860704700BF08ED00E00E2894BF44
:109490004FF4003000207047431E0D2B10B50446DA
:1094A00007D800F007FA20B12046BDE8104000F0D0
:1094B00016BA10BD00F1006000F5003000F07ABB74
:1094C000830705D100F1006000F5003000F0B2BB69
:1094D0000020704700207047014B1868704700BF9C
:1094E0000010005C234B244AF0B51B680446178823
:1094F000C3F30B0056681B0C157AB8422BD0978922
:10950000B84205D101200C2505FB00225668157ACA
:1095100041F20302934220D042F2010293421ED054
:1095200042F2030293421CD041F20102934208BF6F
:109530005A25621E0B46741E0A44934217D214F831
:10954000016F581C7EB92C2482421C7001D9981CD2
:109550005D70401AF0BD0020D5E75925E9E7582590
:10956000E7E75625E5E7034600F8016CE5E718460E
:10957000EFE700BF0010005CBC000024014BC058A6
:10958000704700BF00E8F11F012803D10021024805
:10959000F8F7A0BD704700BF220B04000128014668
:1095A00002D10248F8F796BD704700BF220B0400B5
:1095B000012808B50AD10648F8F788FE80F00100B6
:1095C000BDE80840C1B20248F8F784BD08BD00BF3D
:1095D000220B0400D0E9003283F308881047FEE72D
:1095E0002F4A4FF40030F8B5136800242D4E43F491
:1095F000700313601C222C4B1C725C729A72DC721A
:10960000F8F77EFD2948F8F77BFD0120F7F726F8EB
:1096100020463568F7F722F8254B9D423CD10120C2
:109620002746F7F71BF820463460F7F717F821486C
:1096300000F000FB0546204800F0FCFA1F4B984262
:109640000ED125F0FF021E4B9A4209D1EDB21E2D1C
:1096500006D84FF47A7000274543AC4238BF2C46F9
:109660000820F8F733FE054658B957B1FCF72EF835
:109670000120F6F7F3FF0E4B2C4628463360F6F731
:10968000EDFF02210F48FBF7DBFF20460024FCF72B
:109690006FF8FCF71BF8F8E740F6B8340127C6E787
:1096A00088ED00E050400058AC000024220B04007C
:1096B00007B007B0A0010208A40102085D7D05C53E
:1096C00000ECC2924CA20008034B1B685843034BAA
:1096D00020F07F4018607047D400002414E000E0C0
:1096E000021E054B05480CBF0821012102F00402AF
:1096F00019600421F6F7CEBFD400002410E000E08A
:10970000012200210148F6F7C5BF00BF10E000E0CC
:1097100000220121034808B5F6F7BCFF024B0022E6
:109720001A6008BD10E000E018E000E0022200210D
:109730000148F6F7AFBF00BF10E000E000220221B1
:109740000148F6F7A7BF00BF10E000E0042838B5D5
:1097500005460C4613D80120F6F742FF032D094BAE
:109760004FF000000CBF24F0FF01002153F825301A
:109770001943054B1960F6F733FF002038BD4FF051
:10978000FF30FBE774A2000850400058012804464F
:1097900008B502D10021FFF7D9FF2046F7F73DFABF
:1097A00000F0DAF9436803F110010A68D207FCD42B
:1097B000DA68D20705D5034A5A6002F18832436855
:1097C0005A60704723016745084B9A6882420AD85D
:1097D00002F50012824206D9054A916881428CBF87
:1097E0001846104670470020704700BFD80000247C
:1097F000EC00002420B40D46406811461A46284467
:109800005DF8045BF6F746BF012300220C21FFF749
:10981000F1BFFFEC38B50546BFF34F8F074C6B68BF
:109820001B6913F0070307D00120F6F748FF013C3E
:10983000F5D16FF00F0038BD1846FCE7404B4C00E7
:1098400038B5FFF7C1FF054650B1FEF7C5FE041E4F
:1098500004DB2846FFF7A6FFFEF7D4FE204638BDFE
:109860006FF01204FAE738B5FFF7AEFF054658B1BE
:10987000FEF7B2FE041E05DB2846FFF7C5FF2846AB
:10988000FEF7C0FE204638BD6FF01204FAE7B0F5CF
:10989000803F10B504460AD200F580004001FFF772
:1098A00093FF03698068E41A00EB441010BD4FF089
:1098B000FF30FBE7B0F5803F08B50DD2FFF7E7FFBB
:1098C000002300F1200201780130FF2918BF013385
:1098D0008242F8D1184608BD6FF00D00FBE7F8B5DD
:1098E0000F2800F5806604464FEA46465ED83046AB
:1098F000FFF76AFF0546FEF76FFE002849DB2846A2
:10990000FFF788FF0746002847D12846FFF74AFFA0
:1099100004233A460C21FFF76DFFEB684FF47062A9
:109920000C21E31A28461B0203F4E063FFF762FFF1
:1099300080233A460C212846FFF75CFF2846FFF7B4
:1099400069FF044630BB034604220C212846FFF77A
:1099500051FF23464FF470620C212846FFF74AFF5F
:109960002846FFF751FF2846FEF74CFE0CBB304659
:10997000FFF72AFFE8B106F500352846FFF724FF78
:10998000B8B1AE420CD1002C14BF6FF004004FF4FC
:109990000030F8BD6FF00404E2E76FF00404E2E782
:1099A00033680436013318BF0134EAE76FF00D0065
:1099B000EFE76FF00400ECE72DE9F84F06460F469D
:1099C0001546FFF701FF0446002800F0C2808368B7
:1099D000B34200F2BE80AA1903F580139A4200F246
:1099E000B880FEF7F9FD002865DB2046FFF712FF7F
:1099F0008046002840F0AA8020462037FFF7D2FE9C
:109A0000302325F01F0B0C211A46B946FFF7F2FE52
:109A1000B3444246B04602230C212046FFF7EAFE3B
:109A2000D84532D0BFF34F8FBFF36F8F59F8203C2A
:109A3000C8F8003059F81C3CC8F8043059F8183CF4
:109A4000C8F8083059F8143CC8F80C3059F8103CE4
:109A5000C8F8103059F80C3CC8F8143059F8083CD4
:109A6000C8F8183059F8043CC8F81C30BFF34F8FC1
:109A7000BFF36F8F2046FFF7CDFE08BB636809F187
:109A800020091B6913F0C06F17D0002302220C219C
:109A90002046FFF7AFFE4FF0FF330022142120468F
:109AA000FFF7A8FE2046FFF7AFFE002D41D120466C
:109AB000FEF7A8FD2846BDE8F88F08F12008AFE7BB
:109AC0006FF00405EEE74FF0FF330022142120462B
:109AD000FFF790FE326857F8203C9A4233D1726803
:109AE00057F81C3C9A422ED1B26857F8183C9A425B
:109AF00029D1F26857F8143C9A4224D1326957F8B8
:109B0000103C9A421FD1726957F80C3C9A421AD104
:109B1000B26957F8083C9A4215D1F26957F8043CEB
:109B20009A4210D1636820371B6913F0C06F0AD1C5
:109B300020365E45C7D14FF0FF3300221421204666
:109B4000FFF758FEB3E76FF00405F4E76FF0040584
:109B5000ADE76FF00D00AEE70449054B0A6802F46B
:109B6000E06213430B60BFF34F8FFEE70CED00E0A4
:109B70000400FA052822FF21FAF76CBE10B5054C47
:109B80002046FFF7F7FF04F12800FFF7F3FF024B31
:109B9000636010BDEC1300240000020800F108010E
:109BA000202208B54068FFF769FC202808BF002084
:109BB00008BDFFEC1D4A20F01F0310B554689C42FD
:109BC00025D0D46AA34224D10123282404FB0323F3
:109BD000C0F3820413B93CBB154BD062A01C934266
:109BE00043F820101FD1F4B91A68072A1BD19A6ACA
:109BF000013210D003F128042046FFF7CFFF50B107
:109C000020464FF0FF34FFF7B5FF204610BD00237C
:109C1000DBE70023DCE70548FFF7C0FF0446034805
:109C2000FFF7A8FFF1E71C600024EEE7EC13002427
:109C30001414002438B5144B20F01F02056859682D
:109C400091421AD0D96A8A4215D101222824C0F340
:109C500082000A2104FB023401FB02029C4202F151
:109C6000020253F8225006D0072804D12046FFF7FD
:109C700095FF20B1ED43284638BD0022E6E7204697
:109C8000FFF778FFF7E700BFEC1300242A17002442
:109C900061726D76372D6D2F61726D5F68617264D0
:109CA0006661756C742E630049646C652054617341
:109CB0006B00FFEC0000000000000000B003002477
:109CC00001000000BC03002405000000BC030024C8
:109CD000050000009C03002400000000D0030024C5
:109CE00001000000D803002400000000C803002485
:109CF00000000000626F6F746C6F616465725F6D6D
:109D000061696E004170704272696E6755700069DA
:109D100072712F6972715F756E65787065637465B5
:109D2000646973722E63003C6E6F6E616D653E00F8
:109D300001000000E918000802000000E91800080E
:109D400003000000E918000806010000CD18000813
:109D500007000000CD18000808010000C91800081D
:109D60000A000000E918000809010000E9180008CD
:109D70000B000000E91800080C000000E9180008BA
:109D80000D000000E9180008736572636F6E3A3ABF
:109D9000204552524F523A20416C726561647920DD
:109DA000636F6E6E65637465640A00736572636FDA
:109DB0006E3A205265676973746572696E672043F5
:109DC00044432F41434D2073657269616C20647276
:109DD000697665720A00736572636F6E3A20455248
:109DE000524F523A204661696C656420746F20635B
:109DF000726561746520746865204344432F414354
:109E00004D2073657269616C206465766963653A9B
:109E10002025640A00736572636F6E3A2053756380
:109E20006365737366756C6C7920726567697374AA
:109E30006572656420746865204344432F41434D37
:109E40002073657269616C206472697665720A00BC
:109E5000000002580004025800080258000C025882
:109E6000001002580000000000000000001C025812
:109E70002F6465762F747479537800FF000000001A
:109E800000000000000000240000000000000000AE
:109E9000000000000000000000000000292A000867
:109EA000C12A00089D29000881290008C12800084E
:109EB000112800082B28000865280008C12900087F
:109EC0007128000879280008B5280008B52800087E
:109ED000F92C0008692D0008A12D0008BD2E0008EE
:109EE000B12D0008BD2D000800000000A52C0008C1
:109EF000F9310008A32E00089D2E000871310008DA
:109F0000732E000879330008556D656D00FFECC2B3
:109F1000000000000000000032000000010000000E
:109F20004B000000020000006E0000000300000073
:109F300086000000040000009600000005000000FC
:109F4000C8000000060000002C010000070000000F
:109F50005802000008000000B004000009000000E2
:109F6000080700000A000000600900000B00000064
:109F7000C01200000C000000802500000D00000051
:109F8000004B00000E000000009600000F000000D3
:109F900000E100000110000000C2010002100000FA
:109FA00000840300031000000008070004100000F4
:109FB00020A107000510000000CA080006100000DC
:109FC00000100E000710000040420F0008100000B3
:109FD000009411000910000060E316000A10000050
:109FE00080841E000B100000A02526000C1000002D
:109FF000C0C62D000D100000E06735000E100000F7
:10A0000000093D000F100000696E66006E616E0071
:10A01000286E756C6C2900FF0080E03779C33143EE
:10A0200000003426F56BFC420000901EC4BCC64202
:10A03000000040E59C309242000000A2941A5D426C
:10A04000000000E876482742000000205FA0F241AF
:10A050000000000065CDBD410000000084D78741AD
:10A0600000000000D01253410000000080841E4117
:10A0700000000000006AE840000000000088B340D3
:10A080000000000000407F40000000000000494048
:10A0900000000000000014409A9999999999B93FDD
:10A0A0007B14AE47E17A843F2D431CEBE2361A3F26
:10A0B0003A8C30E28E79453EBC89D897B2D29C3C2E
:10A0C00033A7A8D523F649393DA7F444FD0FA5329F
:10A0D0009D978CCF08BA5B25436FAC642806C80AED
:10A0E0000000000000002440000000000000594073
:10A0F000000000000088C3400000000084D79741A2
:10A100000080E03779C34143176E05B5B5B8934673
:10A11000F5F93FE9034F384D321D30F94877825A3F
:10A120003CBF737FDD4F1575050000002C002F64C8
:10A1300065762F6E756C6C0000000000000000005A
:10A14000A15D0008A55D00080000000000000000FF
:10A15000A95D0008000000000D600008BD66000851
:10A16000AF5E0008AD6100080000000069640008EF
:10A17000E1600008000000002F6465762F74747998
:10A1800041434D256400FFEC85700008C16F000855
:10A1900081720008796F00081769000807690008D4
:10A1A000B1680008C3680008C56800086574000845
:10A1B000FB6C000800000000676B00080000000056
:10A1C000FB6A000800000000E56C000800000000C9
:10A1D000C968000842756C6B00486F6C7962726FD9
:10A1E0000050583420424C20486F6C7962726F20C6
:10A1F0004B616B75746548377632001201000202BC
:10A2000000004062315000010101020301FFECC275
:10A21000CB770008CB77000800000000BB77000870
:10A220000000000025732F257300FFECC981000892
:10A2300065800008A37F000800000000AB800008D4
:10A24000877F000800000000000000002F64657692
:10A250002F74747941434D300053544D33323F3F96
:10A260003F3F3F3F3F0053544D333248375B347CD0
:10A27000355D78000000000007B007B0020007B0AD
:08A28000000008B0263A09B005
:08A2880048EEFF7F0100000019
:10A2900000000000000000000000000000000000BE
:10A2A00000000000000000000000000000000000AE
:10A2B0000000000000002C019C0B002400000000A6
:10A2C00000005802440900249C9E0008000000245D
:10A2D000000000000000000000000000000000007E
:10A2E00000000000000300080000000000C20100A0
:10A2F00037000000000E270700480040387C0900A6
:10A30000397C090000000000FFFFFFFF10A20008D9
:10A310007C00002401000000FFFFFFFF00000000A0
:10A32000000000000000000000000000010000002C
:10A330002CA2000800000000000000001D04000026
:10A340000000000000000000E0010000000000002C
:10A3500059A200083F0000005004000066A2000857
:10A360003F0000000100000001000000002000523A
:10A3700000000008000000000000000001000000D4
:10A3800000210052000010080800000000800000BA
:0400000508000000EF
:00000001FF
